:020000041100E9
:103000000023F7B52E4D2F4C280063616374022610
:1030100001F070F94021FE22217428002A4B00960D
:1030200001F0BAF900283AD1217CFF222800274B71
:10303000009601F0B1F9002831D1254BA2899A42BE
:103040002AD1E389234A934211D1234B6361234B55
:103050002268002A07D1002B05D019002200C1C91F
:10306000C1C21B7B6374280001F082F9F7BD1C4AC2
:10307000934201D00023EBE71A4B1B4A1B68934293
:1030800006D9C02304222800217C9B0001F0FAF914
:10309000164B6361164BDBE700232374EAE7CC236E
:1030A0003821AC2228009B01217401F0EBF90028A3
:1030B000F2D1104B6361104BE381104BC8E7C0465F
:1030C000D441FF1FA061FF1FAC61FF1FAE61FF1F56
:1030D00059590000830500002541001150BD001121
:1030E00082150000C461FF1F87130000D941001141
:1030F00060BD001171410011AAAAFFFF40BD00117F
:10310000F7B5164B0192C318021D002000938823C7
:103110005B05D3181B685C1C1AD09CB2402C18D8D5
:103120008D781E0CAC466746CD782D023D43AE42ED
:1031300006D1019800280ED110000C70240A4C70A2
:1031400003249BB20733A343D218009B9A42DED3D9
:10315000FEBD4432F9E71000FAE7C046FC0F00005C
:10316000802213B503000324019189B25201073173
:103170009B18A14304305A1A88235B05C3181B68A7
:10318000591C03D190429241104016BD99B240297A
:1031900007D80B000733A343C0189042ECD300209C
:1031A000F3E74430F9E7134B134A1B68126810B574
:1031B000FA24934201D81A00F824104BE4021B6849
:1031C0009A4210D813000E4A12689A420ED3013365
:1031D00007D1F823DB029C4203D10A49054808F0D5
:1031E0004BFB200010BDFC24E402ECE7FE24E402CB
:1031F000F7E7C04600C0071100D0071100E0071133
:1032000000F00711FFFFFF7FF0B59BB015000490A1
:103210000391402A00D9A0E006AB59801A80FFF73D
:10322000C2FF0400042816D9002206A9FFF768FF90
:10323000052810D906AB1B88AB420CD1002D07D056
:10324000514B2A000499C01808F0E6FA002802D170
:1032500001201BB0F0BD06AB1D8020000699FFF7D2
:103260007FFF041E7BD1069B0793FFF79CFF802303
:103270005B01C618802307001B039E4201D3F8267A
:10328000F60288235B05F31801931B68013302D013
:10329000019808F031FB3D49019808F0EDFA3B1D1B
:1032A0000293331D05938822029B52059B181B68CD
:1032B00008935A1C3CD044219AB20091402A04D869
:1032C0000320D11D814389B2009103991B0C8B42CD
:1032D00024D0402A22D80122300008A9FFF710FF8D
:1032E000021E1BD1380008A9FFF70AFF04000428BA
:1032F00031D9009A059B9B1880225201B218934243
:1033000040D288235B05C118009A09A808F05CFA2E
:103310001D4B009A09A9F01808F0DEFA009A029BEA
:103320009446634402931A4B029AFB189A42BAD30A
:1033300088235B05FC1821680198013908F09CFA84
:10334000200008F0D9FA039A07AB5A803000079999
:10335000FFF706FF0400002C03D1002079E70428C2
:10336000FBD988235B05E018069908F085FA03234A
:10337000EA1C9A4300D16BE7034B0499E01808F06C
:10338000ABFA65E70424ECE704000011FFFFFF7FC0
:10339000F80F0000F7B505001400402A21D80027D7
:1033A00001AE71803780FFF7FEFE042816D93A007F
:1033B0003100FFF7A5FE042810D93688BC420BD097
:1033C000BD4209D0221CB44200D9321C064B92B235
:1033D000C118280008F0F8F930B2FEBDC04300B2B1
:1033E000FBE703204042F8E70400001137B5042250
:1033F00004000D0001A81649FFF7CCFF02000428C5
:103400000BD1019BA34208D3AB4204D0104901A8C1
:103410000195FFF7F9FE01203EBD0E4C2368200008
:10342000019308F069FA019920000139019108F02F
:1034300023FA80235B01E418074B9C42EED104225F
:10344000034901A80195FFF7DFFE0020E4E7C0462D
:103450005555000000C007110000081130B589B0B3
:1034600008F0FAF910226946254808F01DFB254BA3
:10347000009A9A420ED1019B029A0F2B33D8002159
:1034800001240698013B08D2002900D00292029B39
:10349000013331D10023029325E0551CF2D1020003
:1034A0002100EFE710341022200004A908F0FCFAF4
:1034B000029B013301D1069B0293882304995B058B
:1034C000C918059B06981A03120B049105928142B4
:1034D00003D02B4201D108F077F9019B013B019306
:1034E000019B002BDED1029B002B03D00493049898
:1034F0004168084709B030BDE025014C2D03EFE7D6
:1035000000000111504859368022F8B5964C974B6F
:10351000D200002120001C6008F066FB2300944AC2
:1035200088331A60934B1A786A23002A00D011332B
:10353000E3620A232365904B37221B780820A3639C
:103540008E4B2118E361102323628D4B3B25636171
:10355000C823DB00A36123008C331A602823013ABF
:10356000E26320646364CA67043A211DCA672100CC
:10357000BC310D602100C03108602100C4310B60F6
:1035800021000635CC310D602100083DC8310D60A9
:103590002100D0310A602200D43210602200D832DB
:1035A000136022000227E032210017604222DC3142
:1035B0000A6021001B3DE4310D602100E831086004
:1035C0002100EC310B6023000521F4331960230046
:1035D000F0331A602300183290331A6023009433BA
:1035E000186023001E3A98331A60AF23DB00236073
:1035F000644BFA262363644B644DE360644BF03103
:10360000A3642300FF31FC33B600A16021611E607A
:10361000A5627325E5656D3D6565A56596255D4AE1
:10362000AD00E264666258606766A56600270925FA
:10363000A767E566584F594D606720002567E26728
:103640003A6015279C30676007001A203860200018
:10365000A0300700212038602000A83007004C4827
:1036600038602000F830066026006427A4363760F2
:1036700026005F3FAC3637602600033FB036376028
:103680002600C637B436376026000027B8363760C4
:1036900038269E60424E96205E64424E5A66DE6137
:1036A000414E9A645E62F53EFF3E9E621E269A6718
:1036B000354A8000DE661F675F67DD651D6618623C
:1036C000DA67BE23394A5B00E250394BD8382350C1
:1036D00004302250C4225200A350C623E4205B00D1
:1036E000E1500433334AE1503349344BD16034491B
:1036F000800019503349E938FF38195032490430F5
:10370000195032493248D16132491163324951630B
:103710001900F4310860CE20304940001160304972
:10372000195019002F48F83108602F49D1658221BE
:103730002E4A89005A501A002D490832D1671A00C2
:103740002C49B432116088212B4A89005A501A0042
:103750002A49883211602A4ADA6408F0C5F8012043
:1037600007F0F2FFF8BDC0460004FF1F4464FF1FCE
:10377000106FFF1F1044FF1F4A0AFF1F3A07000087
:1037800080C3C9019A020000DC0500006A1800002D
:1037900050C3000088130000F009FF1F204E0000F6
:1037A0006509FF1F68100000C409000040420F00B7
:1037B00010270000FC00FF1F791CFF1F0000FF1FE7
:1037C000CD2CFF1F5530FF1FED2EFF1F3920FF1F8F
:1037D0002927FF1F5520FF1F0122FF1FC51FFF1FA5
:1037E0004D29FF1F352AFF1F9119FF1F5928FF1F61
:1037F0007D25FF1F8925FF1FC51EFF1F7D1FFF1F82
:103800003D1EFF1F0223F0B50124604D604E2B705A
:10381000604B91B01C70604F03933368002120000F
:10382000FB7006F005FE200006F0FCFC0023984229
:1038300005D0FA78552A02D0332A00D099E03360B7
:10384000042006F05DFF07F0DFFEFFF75DFE08F0E5
:10385000F3F81F2201240021504B10AE1A70504B78
:103860001C70504B1970504B19689143163A0A431B
:103870001A60602219689143403A0A431A6008F0BE
:10388000D3F908F001F9494B9847C120FF21484B73
:1038900080001A588A431A50C522920098588843CB
:1038A000BF39014399509858424908408021C901C5
:1038B0000143802099509958C0050902090A014323
:1038C000995080213C48490108F066F80323220002
:1038D0003A49019400933A4807F0EEFF2C22394907
:1038E00005A807F071FF05AC61782078023406F076
:1038F000B9FCA642F8D1344C344B226803201A405C
:10390000A023DB0213432360802322689B0413431C
:10391000236022682E4B1A4080239B0313432360AD
:103920002C4A2D4B934200D8012008F0CDF808F026
:1039300063F980232268DB0413432360287808F0AE
:1039400003F9039B1878C0B208F04EF808F05CF851
:103950002249042008F0D8F806F09EFE00F040F856
:1039600000F0E6FD00F08EFE00F00AFA002011B033
:10397000F0BD00932100194A042008F0D5F88023F7
:10398000DB059C62FFF76AFD5AE7C0464A0AFF1F43
:1039900034F000401044FF1FD061FF1F480AFF1F92
:1039A000490AFF1F680AFF1FBCF00040E1A20000A7
:1039B00000E100E0FF00FFFF1444FF1F9856FF1FC7
:1039C0001454FF1F68BC001114F00040FF7FF8FF83
:1039D000FFFF9FFF0080FF1F106FFF1F3B000108CC
:1039E000002210B51100112007F01EFE10BD0000CE
:1039F000F8B500230926364F364C3B62E3681120A8
:103A0000B343E36007F0F0FE112008F0A5F81120A1
:103A100007F0AAFE40232268102513432360802369
:103A20006268DB02134363608023A26802211343B0
:103A3000A360A368284A08201340A3608023A268DB
:103A40009B0113430122A360236CAB432364236CCB
:103A50001343236480231B013B62226B1F4B1A40DC
:103A60002263626B1A406263A26B1A40A263E26B2C
:103A70001340E363E3681A4A1340E36006F0F2FB85
:103A80000121082006F002FD8023164A5B00516CDC
:103A900011200B43536407F04FFFFD21C720124B49
:103AA000124A89005A50A36B80002B43A363E3683A
:103AB0000F4A3343E3600F4B195811408022120222
:103AC0000A431A50802292051A600B4B5D63F8BDC1
:103AD00000F000403CF00040FFFFDFFFEFFFEFFF92
:103AE000FFFF7FFF003800400000FF1F5118FF1F3D
:103AF000FF00FFFF00E100E00000054070B5284C2A
:103B0000238C002B23D0228A002A21D1DA002382A1
:103B10006382A382E38223836383A383E38322609C
:103B20006260A260E2601F4D1F4A6420EB809342F6
:103B30000AD8FA220020D200934205D91B4A0A2152
:103B4000981807F019FFC0B200232872238470BDB3
:103B50000720E11CCA7F01320240CA7705D1032544
:103B6000201DC17F01312940C17708325200A35284
:103B7000002321001A00088A01321B180231082A8A
:103B8000F9D1221DD27F9200A350626823689B184E
:103B9000A2689B18E2689B185B099BB2C3E7C0460A
:103BA0001061FF1FB861FF1FB70B000030F8FFFF67
:103BB00030B503A804880B20002C0ED14968074DAE
:103BC00008784978090201430A20A94205D1012158
:103BD00020001980024B1B7A137030BD192A000097
:103BE000B861FF1FF7B5150008AA16884A680F4F7D
:103BF00014785278120222430A24BA4214D10122C4
:103C0000DBB2019200962A0007F096FC041E0BD14D
:103C1000074B1B68002B07D068782A7800021043F6
:103C200042425041013098472000FEBD0229000069
:103C30003C61FF1F30B5012503790400BFB02B4262
:103C400011D00A49408806F0E3FF28420BD0084B08
:103C500001A95B8D4D800B80064B00221B7A60888A
:103C60000B7104F0C7F83FB030BDC0463461FF1F90
:103C70004840FF1FB861FF1F10B50549054806F011
:103C80007DFF0421044A054806F03AFF10BDC046F6
:103C90003461FF1FFFFF000094BC00114840FF1F6C
:103CA00010B5024804F028FF10BDC046353C001195
:103CB000012303700B4B1A7A4270022282709A78A9
:103CC000C270DA780271032242711A7982715A79CC
:103CD000C2710C2202729A794272DB7983720B20D4
:103CE0007047C046B861FF1F022310B50370013B47
:103CF00043700533837010330371443B43712A339F
:103D000083714433C37100230372064B04001B8884
:103D100043720A30FFF7CCFF831D0A30C0B2E37054
:103D200010BDC046B861FF1F10B5142007F0CCFCD1
:103D3000124B14220021186007F056FF002007F0F4
:103D40002BFF012007F0C0FD022007F03DFE0320FD
:103D500004F076F9042006F08BF9052003F0B4FB9B
:103D6000062004F081F8072001F064FA082006F02C
:103D7000A7FE092001F03EF810BDC0464061FF1FBC
:103D800007F0B2FC012007F067FC07F0B5FC00006B
:103D9000094B10B50400984205D0012904D1200038
:103DA000064906F0EBFE10BD0229FCD1013904F0F2
:103DB00061FE0028F3D0F6E7FEFF00006661FF1FFA
:103DC00070B50D7A100004AA2C0016881022144039
:103DD000154220D1002E20D10A78022A18D14A6833
:103DE000517815780E4A09022943914205D00D4AAF
:103DF000914209D01C800A2404E014220A491A8046
:103E000007F0E2FC200070BD0C2208491A80F7E799
:103E10001C800124F6E70824F4E70B24F2E7C046EF
:103E2000F3FF0000F4FF00009C42FF1F7CBD001167
:103E300010B504000749084806F0A0FE074804F042
:103E40009BFD0020E40704D50721054A054806F03C
:103E500057FE10BD6661FF1FFFFF0000913D00117E
:103E6000D8BC00118C40FF1F00B50C4BBFB01A78B6
:103E70000B4902A800F0C0FC6B4680B2D880002835
:103E800009D06A46074B01A91B889380064B002284
:103E9000188803F0AFFF3FB000BDC0464461FF1F6C
:103EA0004561FF1FE640FF1FF041FF1F00B50C4BAF
:103EB000BFB01A780B4902A801F0E2FE6B4680B24F
:103EC000D880002809D06A46074B01A95B8D9380F2
:103ED000064B0022188803F08DFF3FB000BDC0469E
:103EE0006E61FF1F6F61FF1F8C40FF1FF041FF1FBE
:103EF000F7B50E00377A1C0008AB11003D001A8898
:103F000020231D401F423CD13378022B3BD17368E4
:103F10001F785B781B023B431E4FBB4208D01E4FED
:103F2000BB4214D01D4DAB4221D00A252800FEBD56
:103F3000002A2AD1142C2AD82200F06807F044FC69
:103F4000174B1C70012CF1D9FFF7B0FFEEE7002AE8
:103F50001BD1202C1BD82200F06807F035FC114B38
:103F600004211C70104B187807F086FDDEE7E3B2E1
:103F70000124009201940A00310007F0DDFA0500E7
:103F8000D4E70825D2E70125D0E70B25CEE70D259C
:103F9000CCE7C046F3FF0000F4FF00000229000058
:103FA0006E61FF1F4461FF1FF061FF1F332310B5D7
:103FB000040003700A220749013007F005FC064B94
:103FC0000F201B681A0AE37222731A0C1B0E62730D
:103FD000A37310BDB861FF1FE061FF1F30B501255D
:103FE00003790400BFB02B4213D00B49408806F080
:103FF0000FFE28420DD06A46084B02A81B8893800A
:10400000FFF7D4FF6B46D8800022608801A903F037
:10401000F1FE3FB030BDC0466661FF1FE640FF1FA6
:1040200010B5024804F068FD10BDC046DD3F001128
:1040300070B5160004AA148805AA15784A68507845
:10404000117800022A4A0843801805284BD807F047
:10405000ABFD03131E29343F0720032C0BD8042289
:10406000121BAA4200D92A0022491A8030000919DD
:1040700007F0AAFB002070BD0720112CFBD81222EC
:10408000121BAA4200D92A001B491A80EEE707201A
:104090000E2CF0D80F22121BAA4200D92A00174971
:1040A0001A80E3E70720032CE5D80422121BAA425A
:1040B00000D92A0012491A80D8E70720032CDAD841
:1040C0000422121BAA4200D92A000E491A80CDE709
:1040D0000720032CCFD80422121BAA4200D92A00A1
:1040E00009491A80C2E700220A201A80C3E7C046A5
:1040F000DCD5FFFF23BD00118C61FF1F13BD001134
:104100000EBD001109BD001104BD001110B50D2137
:10411000024A034806F0F4FC10BDC046F8BC00118A
:10412000FC40FF1F13B5104C0423217C01AA00F0B2
:1041300061F9002815D16B469A88236852BA92B269
:104140005343228909491B0C9B184B806B46DA8824
:10415000636852BA92B2534362891B0C9B188B80DE
:1041600016BD0120FCE7C046A061FF1FB861FF1F1C
:1041700037B5174C07236A46217C00F03BF900282D
:1041800024D16B461B787F2B20D86B46DD78F0233B
:104190002A041B031A406B469B880E495BBA9BB2EC
:1041A0001A4323682D09534322891B0C9B184B800B
:1041B0006B465A789B7812031B011A4363682A43A3
:1041C000534362891B0C9B188B803EBD0120FCE78A
:1041D000A061FF1FB861FF1F7FB50226154C0022AA
:1041E000217C03AB0096050000F0D6F8002802D031
:1041F000012004B070BD0E23217C0122280000960E
:104200006B4400F0C9F80028F2D16B469A89236804
:10421000D2BA5343228908491B149B184B806B4622
:10422000DA89636852BA92B2534362891B0C9B18B5
:104230008B80DEE7A061FF1FB861FF1F70B5114CD6
:10424000237C002B0FD0382B0ED10F4D280000F00F
:1042500051F8CC23AC222800217C9B0100F012F9FC
:10426000280000F085F870BD084BE2899A42FAD127
:10427000054D280000F03EF800222800217C00F0C7
:10428000E3F8EDE7A061FF1FD441FF1F83050000A5
:1042900070B5144C237C002B1FD06369002B1CD0FD
:1042A000114D280000F026F86369280098470400A3
:1042B000280000F05DF8002C10D10C4B0422995E10
:1042C000002905DA9C801A8801321A80200070BD0E
:1042D000074A9142F7DD9A80F5E70124FEF790FE48
:1042E000F4E7C046A061FF1FD441FF1FB861FF1F64
:1042F0000F27000070B5C17905000C00631E9C41BA
:104300001A4BE402E41849000460C9B2007906F0CF
:10431000F3F8E979687949000131C9B206F0ECF89F
:10432000E8790930C0B207F01FFA0023E366613371
:104330002360AA795B3B002A0ED022689A43023B95
:10434000134323600A23E3610733236200232363BB
:10435000A3630133E36370BD22689A4302231343CE
:104360002360462363610633A361EFE700500040FA
:1043700070B5002504000368DD66C0790930C0B25D
:1043800007F032FA2900207906F052F82900607906
:1043900006F04EF870BD0000F8B51E0006AB1D78A3
:1043A000002304681700E366616007F055FA0123F3
:1043B0008022E3662B0027615200013B08D207F000
:1043C000CBFA08200A4A1168002D03D12800F8BD55
:1043D0002261F2E7236F034203D02369013D33706A
:1043E000013613685B1A032BEED90125EEE7C046B0
:1043F0006008FF1F70B51C00002305681600EB66FF
:10440000696007F029FA01238022EB66230052003D
:10441000013B08D207F0A0FA08200A4A1168002CD4
:1044200003D1200070BD2A61F2E72B6F034203D055
:104430002B69013C3370013613685B1A032BEED9EC
:104440000124EEE76008FF1F002370B50468150023
:10445000E366616007F000FA0123E366256107F077
:104460007BFA8020064A80001168636B034205D105
:1044700013685B1A032BF8D9012070BD0020FCE7FC
:104480006008FF1F70B51D00002304681600E36676
:10449000616007F0E1F90123E36626610F33626B87
:1044A0001A42FCD02B0A23611023626B1A42FCD003
:1044B000EDB2256107F050FA8020074A80001168AC
:1044C000636B034205D113685B1A032BF8D90120F3
:1044D00070BD0020FCE7C0466008FF1F70B51E00DD
:1044E000002305681400EB66696007F0B5F9012345
:1044F000A619EB660F33B4420ED107F02DFA8020D7
:104500000A4A800011686B6B03420CD113685B1A76
:10451000032BF8D9012070BD21782961696B1942FC
:10452000FCD00134E7E70020F5E7C0466008FF1F34
:1045300010B5084CE368002B08D18022064B5202CC
:104540001B689B186360054B1B68236007F074F8B9
:10455000A06010BDE061FF1FC8F00040CCF000403B
:1045600070B5184A936A916A9942FBD116498A68D4
:104570009A421FD39A1A8B60144B0126186893B283
:10458000D202D20E4343424300204C681B0A1B193F
:1045900012029B180E4C0A684B60551CA3420CD8A3
:1045A000002801D04B600A600A4A136008680A4B71
:1045B000186070BD581E821ADDE7084A30009B184B
:1045C0002A00EAE700F00040E061FF1F140AFF1F25
:1045D00040420F00C8F00040CCF00040C0BDF0FFEA
:1045E00070B51F4C23793F2B01D93F2323711D4BFD
:1045F00022791A701878C0B207F01EFB18231A49E6
:104600001A4A0B801A4913800B805380A3791949E9
:1046100080200B800C21938001334B43164D191CD5
:104620000001834200D9011C2980D1806379002BCD
:1046300011D101336371237A012B01D80223237234
:104640006279237A0D4853430A21584307F094F9BD
:104650000B4D286070BDA02BEDD9A023EAE7C04622
:10466000D461FF1F480AFF1FEE41FF1FBC43FF1F1D
:10467000EC41FF1FEA41FF1FE841FF1F71020000EC
:10468000C461FF1FF8B519210020FEF7AFFE114CE1
:10469000011E114D09D10C22104BC1CBC1C4280001
:1046A00007F0A2FAFFF79CFFF8BD0C2220000C498E
:1046B000FEF770FE0C2802D0084B43CB43C40C22FB
:1046C00028000849FEF766FE0C28EBD00C220021DA
:1046D000E5E7C046D461FF1FA061FF1F70BD001158
:1046E000FC0C0000F50C0000F0B51D4C8022A54428
:1046F0000400882069465201400507F025F9902200
:1047000012016A441300200032C832C316C816C30F
:104710008023144C144FA6689B033343A3603B6073
:1047200007F0BAF98823A0685B05C01807F0E4F821
:104730000025882329008022A0685B05C018401945
:104740006944520007F0C8F880230135FF355B014A
:104750009D42EED1A6603E60044B9D44F0BDC04634
:10476000FCEFFFFF2C43FF1F9808FF1F0410000001
:10477000F0B5040087B0002825D0684606F064FF35
:104780001B4C022806D106226946200007F044F897
:10479000002816D06946002301250F262F00E25C71
:1047A000013310091030874038002F003240974005
:1047B0003A0002434A610439062BEFD16846FFF7FD
:1047C00093FF07B0F0BD182269460A4807F0BCF80D
:1047D0006A46A300D358013305D01822FF2168464A
:1047E00007F002FAEAE70134062CF1D1E9E7C04606
:1047F0006509FF1F00090011F0B5002504000E0037
:1048000085B0AA4200D186E04B1C087801934B7812
:104810008978377909021943F3783F061B040B4363
:104820001F43039720706570252800D196E033D888
:10483000112813D807F010F969002B012B012B0167
:104840002B01AA00B800B1002B012B012B012B0179
:104850002B012B012B012B0105012501232800D160
:10486000DEE0DB2800D034E1042A00D8ACE01025DB
:10487000052A05D0551F2A003800711D06F0A4FF37
:1048800005223100200006F09FFF2A003900601D3C
:1048900006F09AFF05353EE0562859D010D8332847
:1048A00000D19DE0552839D02628DAD19F4B290028
:1048B000132218001D0007F097F9FEF7A1FB5CE03A
:1048C000712800D177E0722800D180E0602800D103
:1048D0008BE0DC28C5D1022A00D875E07378BFB21E
:1048E0006370B378A370032A05D0033A390092B2FB
:1048F000F01CFEF789FC10223900E01CFEF74AFD8F
:10490000C51C002807DA60705CE00C222000884992
:1049100006F05AFF0C25280005B0F0BD013A854D80
:104920000C2A13D8002A0AD02800019906F04CFF5F
:10493000FFF756FE0C2228007F49FEF765FC290090
:104940000C22601C06F040FF0D25E4E70C22EBE78B
:10495000784D7A4B2A0043CB43C2E9E7013A734DC5
:104960000C2A11D8002A08D00199280006F02CFF43
:104970000C2228007249FEF747FC29001322601C14
:1049800006F022FF1425C6E70C22EDE706226D494A
:10499000601C06F019FF0625BDE712226A49601C5B
:1049A00006F012FF1325B6E708226849601C06F0DE
:1049B0000BFF0925AFE77178F02905D8644B1888FB
:1049C00001F0BAFD0225A6E7FF236370FAE7614B09
:1049D000012A03D072789A706270F3E79B78F4E74B
:1049E0002000FFF7E3FA050095E7013A594B5A4DCD
:1049F000072A10D8002A10D00121280059700199E7
:104A000006F0E2FE01F05CF829000722601C06F0C7
:104A1000DBFE08257FE70722EEE700225A70F3E766
:104A2000042A04D94D4D2F6006F006FEA860FFF75A
:104A300097FD0422039003A9601C06F0C5FE05251E
:104A400069E7474D062A15D906222800019906F084
:104A5000E3FE00280ED006220199280006F0B4FEDD
:104A6000062240492800FEF7CFFB0123394A9178FE
:104A70000B43937029000622601C06F0A5FE072553
:104A800049E7012AA0D07078FFF772FE9AE7012863
:104A900000D0E6E6931E344F132B06D87378002B14
:104AA0000BD100F015F900F04BF9304B39001D78AF
:104AB000601C6A1E06F088FE2DE7551E2A0001992B
:104AC000380006F081FE38002949AAB2FEF79CFBA7
:104AD000E9E7DA281DD1042A00D875E7082A15D994
:104AE000B37972791B021343F27912041A43337AB1
:104AF0001B0613433B603B680522310020000393F3
:104B000006F062FE0422601D03A950E7FE236370D5
:104B1000F1E7DE2800D057E7511E012A01D1002518
:104B2000F9E6019800F0B2FFF9E7C046A061FF1F67
:104B30007CBD0011D461FF1FFC0C000070BD001192
:104B4000F50C0000AC61FF1F8C61FF1F3043FF1F9D
:104B5000F041FF1FD061FF1F8D42FF1FE061FF1F6B
:104B60006509FF1FADAC0000D163FF1FCF63FF1FBE
:104B7000AEDE000070477047020010B5094B0A32E4
:104B8000094C92B2DA815A8298811882207802F018
:104B900039FB0422054B012120781A7006F06CFFC6
:104BA00010BDC046BA42FF1F1A64FF1F1964FF1FE1
:104BB000013870B5042809D806F0F6FF0309280863
:104BC0001200234B0221187806F056FF70BD204BCF
:104BD0000821187806F048FE00221E4B1A72F5E7ED
:104BE000802200241B4B1A4D52001A8108211A689A
:104BF0002878DC7206F090FF2100287806F06CFD22
:104C0000012000F063FE00F05BFFDFE7104B08219E
:104C1000187806F029FE1048FFF766F80F4B104A87
:104C20009B79002093800F4A13808022094B520009
:104C3000D8721A8100F04AFE00F042FF0A4B9B78BE
:104C4000002BC3D0094A136006F05EFDBEE7C046E4
:104C5000F061FF1FC461FF1FF941FF1FD461FF1FF7
:104C6000BC43FF1FEA41FF1FD061FF1F34F000402B
:104C700010B501290BD1012809D1054B1B78002B58
:104C800005D02622034B04485A72FFF775FF10BD6A
:104C9000F263FF1FC461FF1FC40900000300F0B5E9
:104CA0000A4D8E18B14202D152008018F0BD0C7826
:104CB0002F6824093C5D0F271C700C7801313C40A3
:104CC0002F683C5D5C700233ECE7C046E441FF1F97
:104CD0000D22124B10B51A700C23114C1149237080
:104CE000093A033B1048637006F06EFD2D23012244
:104CF0000E490F48A371FFF7D1FF01220D49FFF7BD
:104D0000CDFF01220C49FFF7C9FF030000200B492A
:104D100002001870FEF778FA10BDC046EE63FF1F60
:104D2000CF63FF1F23BD0011D163FF1F6709FF1F62
:104D3000D663FF1F6609FF1F6509FF1FAEDE000077
:104D400070B5134C142220001249FEF723FB431EBA
:104D5000114D132B19D8AB78002B16D0431C2B7098
:104D600009236B7000230019037028780B4B013066
:104D70002900C0B2187006F04FFC297822000139D2
:104D8000C9B2002005F0DAFD70BDFFF7A1FFECE726
:104D9000D163FF1FAEDE0000CF63FF1FEE63FF1F76
:104DA00010B5114B1A781870002A0ED000280BD1BC
:104DB0000E4B1A78062A07D85423D340DB0703D5B5
:104DC0000B4B187802F01EFA10BD0028FCD0074BE0
:104DD0001B78012B02D0033B022BF5D8044B012199
:104DE000187806F049FEEFE7F263FF1F1964FF1F12
:104DF0001A64FF1F70B54A4E4A4A4B493070012071
:104E000005F028FC00F0DAFEFEF7FAF806F00CFDDB
:104E1000032246494648FFF741FF2D2403000422A0
:104E20001C7044490130FFF739FF30230470424DB4
:104E3000424C437083702E3B062220004049EB8792
:104E4000FEF7A8FA062813D0200006F0FDFB022882
:104E500009D00321200006F0AFFC8D23E3706E3BE8
:104E6000237119336371062220003549FEF7CCF90E
:104E7000344B1B68FC335C64FFF762FF0020FFF7D4
:104E80008FFF314C314A0121314B1278207802F0EA
:104E90007BF9304A304B12780021207802F074F907
:104EA00001222E4B1A702E4BDB78552B31D12D4B16
:104EB0003B325A722C4B2D4AAB81EA812B826A829B
:104EC0002021307806F088FE0120404205F082FD66
:104ED0000120404205F01EFEFFF718F9FEF7CCFE58
:104EE00000F0B2FC01204042FEF7A2FF012006F0D4
:104EF000DBFCF02001F004FB0121307806F0BCFD62
:104F0000307802F0DBFA1A4806F09EFEFEF770FDDC
:104F100070BD6422174B5B7953431A000A32CBE70A
:104F2000F061FF1F754B0011714C00113043FF1FE2
:104F30008C61FF1FAC61FF1FBA42FF1F6509FF1F95
:104F4000ADAC00004464FF1F1A64FF1F1842FF1F2E
:104F5000F941FF1FEE63FF1FCF63FF1FC063FF1FF9
:104F6000D061FF1FC461FF1FC4090000CE0900000B
:104F7000F261FF1FD461FF1FF8B50A0020230D0066
:104F80001A40194263D05E4B1B78002B5CD0FFF7B0
:104F9000E7FA5C4B5C4C5D4E99686268737A8A1ADA
:104FA000DB039A4202D36160FEF722FD327A217A56
:104FB000531EDBB2994205D1FFF740F9002000F003
:104FC000B5FD15E09142F9D300272772FFF760F98C
:104FD000A37ABB4202D0A772FEF790FD012000F039
:104FE000A5FD4B4F3800FEF77FFE390006F0B4FBFD
:104FF000637A002B25D0013BDBB26372002B20D1FA
:10500000444BDB78552B01D106F07EFBE37A002B75
:1050100012D00023A27AE3729A4202D0A372FEF762
:105020006DFD3D4A3A4F1388380001331380FEF777
:105030005BFE390006F090FB642370795843FFF75C
:105040009BFD237A0133237220206840F8BD0BB208
:10505000002B0ADA314B187806F0D6FB002801D075
:1050600006F012FB80200002EFE70224214206D066
:10507000254B01201A72FFF793FE2000E5E70B078E
:105080001ED5FFF76DFA1F4B1F49204C98684A68E0
:10509000637A821ADB039A4202D34860FEF7A8FCC7
:1050A000FFF7F6F8FFF7CAF8012000F03FFD00F027
:1050B000E5FB2368DB0701D5FEF7B2FF0820C4E754
:1050C000CB0609D5FEF71AFD0D4B1B78002B01D13D
:1050D000FEF7E6FD1020B8E70124214207D0104872
:1050E00000F06CF806F0B0FC00F006FDC5E7042403
:1050F000080020402142A9D0FEF7B6FEBDE7C04619
:10510000F263FF1FE061FF1FC461FF1FD461FF1F37
:10511000F941FF1FD061FF1FB861FF1FF061FF1F42
:10512000DC41FF1FF0B51B4B1B4F1B883A88040066
:105130001A4E1B4D85B09A420DD832889A420AD336
:10514000184B1A882B889A4205D1174A174B128898
:105150001B889A421BD0052001F028FA3B8802AA3E
:1051600013803388019053802B88114D93800F4B0F
:1051700002A91B88D3800F4B2A78188802F044FFBD
:105180000D4B08212878019A1C7006F0C5FA05B06D
:10519000F0BDC046BE63FF1FEE41FF1FEC41FF1F85
:1051A000EA41FF1FBC63FF1FBA63FF1FE841FF1FF7
:1051B0001A64FF1FF041FF1FB863FF1F13B50C4BAC
:1051C0001C78002C11D1002801D00A4B18600A4A23
:1051D0000A4B11780A4A10780A4A01920A4A009248
:1051E000002205F0A3FA200016BD1124FBE7C046FB
:1051F0001964FF1FB463FF1F1864FF1F0864FF1FBB
:105200001A64FF1FF463FF1FF863FF1F10B5064BFE
:1052100012201B78052B06D1044B13221988044B4E
:10522000187801F09FFB10BD1964FF1FF041FF1FAC
:105230001A64FF1F10B500240122114B524218704E
:10524000104B1C70104B1A8002F038F904220F4BDF
:1052500021001A700E480C3206F0BEFB102221000D
:105260000C4806F0B9FB07220B4B1C600B4B1C7063
:105270000B4B1C700B4B1A700B4B1C7010BDC046B7
:105280001A64FF1F1964FF1FF041FF1F1864FF1FFE
:105290000864FF1FF863FF1FF463FF1FCE63FF1F47
:1052A000CD63FF1FF241FF1FCC63FF1FF8B5174C02
:1052B0000600257806A814240078052D23D1B41FF4
:1052C000134FA5B21824BD421DD88D1FADB2BD42EB
:1052D00019D8FA256D00AA4215D21D000D4F0A3DBE
:1052E000ADB2BD420FD80C4C26800C4C21800C492D
:1052F00000240A800B4A1380FFF714FF0A4B042195
:10530000187806F0B1FA2000F8BDC0461964FF1FF6
:10531000790C0000750C0000EE41FF1FEC41FF1FEF
:10532000EA41FF1FE841FF1F1A64FF1FF0B50BB2EF
:105330000D0089B0002B00DB70E1A44E307806F040
:1053400063FA041E50D00378A22B00D122E1D02BA7
:105350001AD0912B45D143780E2B42D19C4B828899
:105360009A423ED19B4A83681278052A39D103209C
:1053700018567F2835D0984B1B68002B31D05B68BE
:10538000002B2ED098472CE08078072829D806F0EB
:105390000BFC0428183F3F74A8D86378002B0CD16D
:1053A00001218C4B19708D4B1A78002A5BD08C4BE5
:1053B000307801F0E9FE002855D00722854B1A709D
:1053C00051E061780029F8D1E378002B11D0854AAB
:1053D000854B1278307801F0D7FE60706378002B2F
:1053E000EBD1200006F050F980200002684009B09F
:1053F000F0BD784B1B78022BF3D00121307806F0FA
:10540000D3F90028EAD10121307806F035FBE5E731
:105410006378002BD1D16F4F032807D13B78052B40
:1054200002D101333B701EE00223FBE76F4B1A8869
:105430006F4B0293002A0BD01B78002B03D0012165
:10544000307806F069F93B78062B04D1013BE9E797
:10545000029B1A70F7E7042B41D10121029B30789F
:10546000197006F009FB5C4B1B68002BB9D01B6858
:10547000002BB6D0574A107884E76378554F002B3D
:1054800027D10622211D5B4806F09EF962895A4BFE
:105490005A491A80A2895A4B1A80E3890B80052148
:1054A000397058490A80584A1380228A574B1A800B
:1054B000574B1B78012B09D11F2001F077F8FA22F6
:1054C000920042430421307806F026F90022484B2E
:1054D00075E7312B00D070E70022454B1A7003238B
:1054E000A0E706220021434806F076FA0023454A49
:1054F00004211380444A30781380444A138006F014
:10550000B3F90821307806F0AFF9A379083B5A4285
:105510005341304A03331370304B1B78002B06D0B5
:10552000334B30781A78002A06D001F06BFE012246
:10553000314B52421A8096E70121197006F09CFA0D
:10554000F5E70821307806F08FF96378002B00D05A
:1055500047E72C4B2D4F0293E388029A04211380D6
:10556000294B307803932389039A138063893B8006
:1055700006F01AF9002800D033E7264B1B68002BF1
:1055800000D12EE7039902983A88098800881B68A1
:10559000984726E74379132B00D022E70389012B94
:1055A0000AD11D4B1B78022B06D10821307806F05A
:1055B0005BF9FFF72BFE14E7052000F0F7FF082149
:1055C0000200307806F0A8F80BE7C0461A64FF1F07
:1055D000051400001964FF1FB463FF1F1842FF1F6A
:1055E000F941FF1FEE63FF1FCF63FF1FF063FF1F33
:1055F000F263FF1FC163FF1FF041FF1FC863FF1F5E
:10560000CA63FF1FBE63FF1FBC63FF1FBA63FF1F98
:10561000C063FF1FB063FF1FB863FF1F8020C0017E
:10562000014200D0E2E6CB0731D5324B1B78002B8C
:105630001DD0314E05AC3378052B1AD1023B2370B7
:105640002E4B21001B7823722D4B1B7863722D4B40
:10565000187801F03DFD002809D007202A4B307052
:105660001B68002B03D01B68002B00D0984701203B
:10567000BCE60E20254B06221B7825492370254BBE
:105680001B78637002ABC01806F09EF8D8E70223BF
:1056900008001840194209D0174B1B78052B03D17D
:1056A0001D4B188806F028FA02209FE604242142A8
:1056B00003D0FFF737FD200098E6082308001840C4
:1056C000194200D193E6154B1C78012C03D0022C13
:1056D0000DD008208AE6124B124A134913481B8842
:1056E0001288098800880094FFF7E0FDF1E7FFF7D2
:1056F0008DFDEEE7F263FF1F1964FF1FF241FF1FEC
:10570000CC63FF1F1A64FF1FB463FF1FCE63FF1F2C
:10571000F341FF1FCD63FF1FF041FF1FB863FF1F61
:10572000E841FF1FEA41FF1FEC41FF1FEE41FF1F51
:1057300010B502A804880B20002C10D14968087805
:105740004978090201430C48814209D1022119809C
:105750000A4B59881170DB7800205BB2537010BD82
:10576000074C0A20A142FAD102211980034B9988E3
:1057700011705B79F0E7C0466E2A0000B861FF1F28
:105780006F2A0000F7B5150008AA16884A680F4F5F
:1057900014785278120222430A24BA4214D1012208
:1057A000DBB2019200962A0005F0C6FE041E0BD162
:1057B000074B1B68002B07D068782A78000210433B
:1057C00042425041013098472000FEBD02290000AE
:1057D0002C64FF1F30B5012503790400BFB02B42B4
:1057E00025D01449408805F013FA28420CD0124BFA
:1057F00001A95B8D00220B8002234B800F4B5B883D
:105800008B80608802F0F6FA0D49608805F000FA96
:10581000C0070CD50B4B01A91B8800220B8002236B
:105820004B80064B9B888B80608802F0E3FA3FB088
:1058300030BDC0462464FF1F1C42FF1FB861FF1F1C
:105840001C64FF1F7642FF1F10B5074C074920005C
:1058500005F094F92000064905F090F90721054A62
:10586000054805F04DF910BDFFFF00002464FF1F3F
:105870001C64FF1F9CBD00111C42FF1F10B5024895
:1058800003F03AF910BDC046D55700110221430874
:1058900088400B400A31084003430E20024AD17869
:1058A00081430B43D37070478D42FF1F064A137923
:1058B000410705D580210B4380011371907170471A
:1058C0007F210B40F8E7C0468D42FF1F054A537801
:1058D000002803D080210B43537070477F210B4079
:1058E000FAE7C0468D42FF1F0F21114BDA780A40BC
:1058F000DA70502810D901310A43DA702022D978A1
:105900000A43DA704022D9780A43DA708022D978C3
:1059100052420A43DA7005E03C28EFD82828F1D833
:105920001428F3D80122D9780A43DA707047C046A8
:105930008D42FF1FF8B57F23324D04006E789E43E1
:10594000314B984205DD76232B70363B33436B7029
:10595000F8BD2E4B984203DA58232B701433F5E729
:1059600083B21A0000215F32294892B2294F297070
:1059700082422DD9A9708C4203DA5B421CB22023EB
:105980002B70053420B20A2105F0F6FF04B2FA2389
:105990009B009C4233DB80232A785B4213432B70AD
:1059A0006421200005F0E8FF0A2100B205F0ECFFB9
:1059B00009B22A787B5C13432B700A21200005F082
:1059C000DBFF0A2100B205F0DFFF09B27B5C0AE0D1
:1059D0008022AA70002CDADA5B421CB220232B70E2
:1059E0005F23092CE9DC1E430A2120006E7005F0BC
:1059F000CBFF09B2AA787B5C1343AB70A8E7632C9A
:105A0000CEDCEDE78D42FF1F1B4E00001DFCFFFFAB
:105A10002A080000C6BD00117F23F7B5194FCD013C
:105A20003E7904009E433E71EDB2632806DD093BDA
:105A300033433B7140231D437D71F7BD03000933A0
:105A400004DA582333433B716C23F4E70E4B019384
:105A500000280BDA0423444224B23B710A212000BF
:105A600005F092FF019B09B25B5CE4E70928F5DDD4
:105A70000A2105F081FF019B00B21B5C1E433E71B1
:105A8000ECE7C0468D42FF1FC6BD0011F8B50A4FB6
:105A900005003B780E00002B0CD0084C2000FEF7D0
:105AA00029FC33002A0020003978FEF717FD20007A
:105AB000FEF75EFCF8BDC0463864FF1F9442FF1F2E
:105AC00070B50A4E0A4D07223100280005F0A4FEE9
:105AD000002809D0074C31000722280005F074FE89
:105AE00008212000FFF7D2FF70BDC0468D42FF1F86
:105AF0003164FF1F3064FF1F7F2210B50A4B5978B5
:105B00009143033A1A70103A0A435A7078220E21D0
:105B10009A70DA788A43DA7006221A7139325A7129
:105B2000FFF7CEFF10BDC0468D42FF1F10B5002805
:105B300032D01E4C0223E05E1D4B1B685B062CD549
:105B400009233221584305F017FF4130FF3000B2DE
:105B5000FFF7F0FE0520FFF799FE0422A35E154A29
:105B60006320934205DC32331800642105F004FF02
:105B700000B20121FFF750FF207AFFF7B5FE0020A9
:105B8000FFF794FE0C4B1878053843425841C0B2D9
:105B9000FFF79CFEFFF794FF10BD0A21053005F0CA
:105BA000EBFE00B2FFF7C6FE0320D4E7B861FF1F8B
:105BB000D461FF1FDD2600001964FF1F70B50024AB
:105BC000094D2800AC71FEF795FB10233E212800FB
:105BD000064AFEF783FCA04200D13E34044B280065
:105BE0001C70FEF7C5FB70BD9442FF1FB6BD0011CF
:105BF0003864FF1F0200F0B501270A480A4E511809
:105C00008B1A002B00DCF0BD08241578430868408F
:105C100038404000805B013C58406D08002CF5D1B5
:105C20000132EDE7FFFF0000D6BD0011F0B5002501
:105C30000F269D4200DBF0BD4C5D07094440344017
:105C4000A400A05801357840F3E70000F0B589B012
:105C50006A460D000B000F27110010351C78013328
:105C6000260024093E40167054700232AB42F5D132
:105C70002023024AFFF7DAFF09B0F0BDDCBD0011B6
:105C8000F0B54E780B7889B036020C001700019001
:105C90001E43012A61D9954B9E4200D877E001331B
:105CA0009E421CD1062A17D1CA788B7812021A4359
:105CB0000B791B0413434A7912061A438C4B5A6121
:105CC00000221A705A808B4A5A608B4A9A608B4A1B
:105CD000DA60002009B0F0BD88225205EEE7884B5B
:105CE0009E423CD182498B78002B00D0F6E00C2AF2
:105CF00031D10F22A3789343E27812021343227921
:105D0000120413436279120613434B60E279A079BF
:105D100012020243207A00041043627A1206024300
:105D2000CA60E27AA07A1202024376484A8183422C
:105D300008D804236E49142201980B7005F044FD25
:105D40001420C7E71201D21889235B059A42F0D8C4
:105D500001238B70BDE7022AFAD00523EAE76A4ADD
:105D600001239642E6D1FFF751FA052F0CD9E378CB
:105D7000A2781B021343227912041A4363791B068B
:105D80001343624A0393136005F0BEFCA1E7584D2C
:105D90002B78002B9DD1AB78002B00D1A0E02B8974
:105DA00001339BB20093B34200D091E0132AD4D9BF
:105DB000CF7C8B7C3F02122120001F43FFF71AFF8C
:105DC000874200D08EE0002E3DD1E378A2781B02FE
:105DD00013432279E96812041A4363791B061343BB
:105DE00003930A228B4212D1FF23A370E370237125
:105DF00063716B89002B09D1E37B227C1B021204A7
:105E00001343A27B13431B0901336B8100226B896F
:105E1000002B8ED0002A67D1686837013818000B34
:105E20006B6900030390984205D9686105F064FD31
:105E3000EB780133EB7068681022A11C381805F06C
:105E40004BFD2E8145E76F89009A7B1E9BB29342E2
:105E50003AD1E278A37812021A43237905A81B04E9
:105E6000134362796C6812061A43EB68009203923E
:105E7000211D0C22049305F0A7FC0120260004A993
:105E800040421036FFF7E2FE013F012F17D1009A82
:105E90000B232861824200D04CE704221C492000D9
:105EA00005F01AFD042203A9686805F04DFDE968B4
:105EB000039AFF23914200D13CE7F73B3AE73100D8
:105EC000FFF7C4FE1036DFE70923B742A4D831E755
:105ED000009BB34200D9FCE607232BE7022329E706
:105EE000032327E7062325E70A2323E7FFFE000015
:105EF0009C42FF1F00000111FFFF0000504859366F
:105F000001FF0000FFFF001102FF000034F000401D
:105F1000A842FF1F10B5034C0B000122210000F026
:105F20006BFA10BDD56000110B8870B506000D002E
:105F30000224162B11D92B000322094900F05CFA28
:105F4000041E0AD1074B2A881B88191C934200D9CA
:105F5000111C300089B200F0EFFA200070BDC0467D
:105F6000016100114A64FF1F10B54A780400013A2C
:105F70000B000220012A07D80A78002A04D0052243
:105F80002000024900F038FA10BDC0462F61001110
:105F90000A7810B50B0004000220002A04D0072262
:105FA0002000024900F028FA10BDC046DB61001154
:105FB0000A7810B50B0004000220002A04D0092240
:105FC0002000024900F018FA10BDC04641620011DD
:105FD00010B5034C0B000B22210000F00DFA10BD90
:105FE0007162001110B5034C0B000D22210000F06E
:105FF00003FA10BDE362001110B5034C0B000F2231
:10600000210000F0F9F910BD3D6300110A7810B5C8
:106010000B0004000220002A04D0112220000249B3
:1060200000F0EAF910BDC0464D630011002310B521
:106030001322190000F0E0F910BD000010B5034C68
:106040000B001722210000F0D7F910BD9F6300114B
:10605000002310B51922190000F0CEF910BD000080
:1060600010B5034C0B001B22210000F0C5F910BD38
:10607000D9630011F7B584890D0006000121002CB9
:1060800022D000238268D3561778002B1EDA0C2CFE
:106090001AD90C3CA4B2131940880093230002F0D3
:1060A00086FE431E984101307B06DB0F6B703F2359
:1060B000013C1F40A4B22870AF70AC80002C07D008
:1060C000B3680133AB6000210800FEBD0020EBE7A0
:1060D000AC60F8E70B7803704B8843704B881B0A61
:1060E00083700B79C370042070470420022B06D103
:1060F0000020537811781B02009A0B4313807047DD
:106100000B8803700B881B0A437002207047042021
:10611000009983420AD1537810781B0203430B8005
:10612000D37890781B02034300204B807047F8B56A
:106130000D004B7801240021461C03702B788B4204
:1061400001D82000F8BD6B78B01C4F1C012B10D17A
:10615000890069184B88022233704B88B9001B0AEA
:106160007370691805F048FC04360434A4B2F9B21F
:10617000E4E7122359436B185A88043132705B8864
:1061800010221B0A7370691805F036FC123612349F
:10619000ECE770B5049D14001E00052B01D8042007
:1061A00070BD637812781B0213432B80E378A278CA
:1061B0001B02134302226B802A71211D681D063EBB
:1061C00005F01AFCB2B22A81E92AE8D82800A11DFC
:1061D0000A3005F011FC0020E2E7002310B50A7830
:1061E0009A4201D8900010BD9A008A185488013351
:1061F00004705488DBB2240A4470948884709288B6
:10620000120AC2700430EAE710B51100029C062B96
:1062100004D004201022142B01D010BD02222271C0
:106220004B7808781B0203432380CB7888781B02C5
:10623000034363800431601D05F0DEFB0020ECE7C2
:1062400010B50C788B7804315C43E4B20370220003
:10625000013005F0D1FB601C10BD0420022B06D1DB
:106260000020537811781B02009A0B43138070476B
:1062700010B50C000A88023105F0BEFB208810BD65
:1062800070B504000D0004981100012B01D8042002
:1062900070BD167852781202324302800200F13249
:1062A00055701470E125002C00D10C35023B9AB2D8
:1062B0004280AA42EBD80231043005F09DFB002059
:1062C000E6E70420009983420AD1537810781B0234
:1062D00003430B80D37890781B02034300204B804C
:1062E000704710B50C000A88023105F085FB208844
:1062F00010BD000070B501211E000420049C0E405A
:106300000B4218D1CB40DDB28D4214D90A49DBB221
:10631000098899420FD32300EE331D7033005800D3
:1063200011184978165C0902314301332152D9B260
:106330008D42F4D8002070BDB442FF1F10B50C0090
:106340000A88023105F058FB208810BD10B50C7882
:106350008B7804315C43E4B203702200013005F015
:106360004BFB601C10BD10B511000298032B01D827
:10637000042010BD14785278043B1202224302809C
:10638000CA788C781202224342809AB28280EB2A29
:10639000EED80431063005F02FFB0020E9E710B5F8
:1063A0000C000B8803700B881B0A43704B888370AA
:1063B0004B881B0AC3708A880430063105F01CFB29
:1063C000A088043080B210BD0420012B03D100202E
:1063D0001378009A1370704710B50C000B88037087
:1063E0000B881B0A43704A880230043105F004FB15
:1063F0006088023080B210BDF0B589B003931E4BA7
:10640000029242000700D05A019102F020F81325B1
:10641000061E2DD0029B01240370019B002B04D08B
:10642000001903999847001984B26B461B7A5BB236
:10643000002B0FDA1021380002F01CFB1925002870
:1064400013D130003219E1B202F066FC051E0CD106
:106450000C34A4B2042304AA380005A9938006963C
:10646000948101F0AFFD051E02D0300005F064F903
:10647000280009B0F0BDC0464864FF1F70B5050094
:106480000C0000280CD00020814209D010222000EE
:10649000044905F0B1FA01202B7823736B786373FC
:1064A00070BDC0461CBE0011F0B506000D001700FF
:1064B0001C0085B002291BD00020102907D1022B17
:1064C00007D0102B03D115E00020102C08D005B008
:1064D000F0BD69463800FFF7D1FF2A0069460BE09E
:1064E00069463000FFF7CAFF22006946380004E021
:1064F000022BE9D12A003900300005F01DFBE6E748
:10650000031CF02800D9F023032008499AB2013A6D
:106510000B80D317034006499B189B100B80D30FA9
:1065200004499B185B100B807047C046B842FF1FA0
:10653000B642FF1FB442FF1F034B1B888B4202D39E
:10654000024B4000C1527047B842FF1F4864FF1F12
:10655000014B4000185A70474864FF1F1722014B37
:106560001A8070474864FF1F70B505000E2005F0C3
:1065700003F9041E13D0D023037000230622837076
:1065800007494570033005F037FA064B2100DA8AD7
:1065900062811B7E2373044B187805F005FA70BDE9
:1065A0006464FF1F5464FF1F0843FF1F262803D89D
:1065B000024B4000C05A70470148FCE7BA42FF1F37
:1065C000FFFF000070B506000C00094D1C220021E1
:1065D000280005F001FA074B1E70074B1C7005F0F0
:1065E0000BF90123002801D0002312202B7070BD6D
:1065F0005464FF1F0843FF1F7564FF1F70B505003B
:106600000D4C0800E260A16010220021656005F0D9
:1066100023FB012803D11021A06802F058FD1022AD
:106620000021280005F018FB012803D11021606823
:1066300002F04DFD70BDC0465464FF1F70B5041ECE
:1066400005D1002903D006220D4805F0D5F90D4BE0
:106650001D78012D11D1002C05D102221A7005F0F0
:10666000EBF8280070BD00221A70074B1B78FF2B37
:10667000F7D02000FFF778FFF3E70025F1E7C046E9
:106680006464FF1F5464FF1F0843FF1F030010B51D
:10669000002801D1002010BD00780B4A002803D14A
:1066A0005988D1821B7913761378022BF2D10023FB
:1066B000984200D103331370044B1B78FF2B01D099
:1066C000FFF752FF0120E6E75464FF1F0843FF1F56
:1066D000002911D000280CD04B79012803D1402289
:1066E0005242134303E03F221340032802D001200B
:1066F0004B7170474022F4E70800FAE770B5094D86
:106700000100287800280BD0074C0622200005F055
:1067100073F921002878FFF7DBFF200005F054FA19
:1067200070BDC0467464FF1F4E64FF1F00290AD06D
:10673000012808D13F224B799343C02B03D0403B23
:106740005A425341981C704770B5174D06002B787C
:10675000FF2B15D00A2005F00FF8041E10D0D0230F
:106760000370C83B8370114B11491B784670C3708E
:106770000622043005F040F92100287805F014F9CC
:106780000C4B1B78012B0DD10B4B1B68002B03D03E
:106790009B68002B00D09847084B04211878084AC2
:1067A00005F0BAF970BDC0460843FF1F7464FF1FAF
:1067B0004E64FF1F7064FF1F9C64FF1FA064FF1FD7
:1067C00060EA0000014B98687047C0465464FF1FA0
:1067D000014BDB68186870475464FF1F074B10B506
:1067E000DA68136801331360054B1878FF2803D06B
:1067F0008021C90105F040F910BDC0465464FF1F57
:106800000843FF1FF7B50E0002F0C8F8051E1CD0A4
:106810000E4B06621F78002F00D10778AB7910204D
:10682000019304F0A9FF041E0FD0D0230380C73BBF
:106830008370019BE91DC3700622043005F0DCF86B
:1068400021003800E66005F0AFF8F7BD0643FF1FF2
:10685000014B18787047C0467464FF1F054B002831
:1068600005D1054B1A78054B002A00D1014B1800C1
:106870007047C0466464FF1F7464FF1F4E64FF1FAF
:10688000014B58687047C0465464FF1F024B18689C
:10689000431E9841C0B270477864FF1F421E030038
:1068A0000120152A03D9FF3B5A425341D8B2704701
:1068B000F0B51C0000230E0085B0039002920B700F
:1068C000029A934201D3002019E0E55C5A1CD2B22F
:1068D000002DF8D0029851198142F4DC0233DFB266
:1068E000A35C18000193FFF7D9FF002807D0013DF2
:1068F000019A0399EBB233708A4202D1E01905B0D4
:10690000F0BDDB19DBB2DBE710B50C0002F09EF83E
:1069100003001220002B03D02100588804F0A4FEAD
:1069200010BD000070B50E4D84006359002B15D0CA
:10693000186A002801D004F0BFFE2B59586A0028BD
:1069400001D004F0B9FE2B59986A002801D004F058
:10695000B3FE285904F0B0FE00232B5170BDC04691
:106960008464FF1F1C4B70B504000E001500994293
:106970000AD11A4B1B68002B01D1122070BD1B6875
:10698000002BFAD09847F9E7154B994215D1134BD4
:106990001B68002B0AD01B68002B07D098470028E3
:1069A00004D1104B1C70104B1D70E7E7290020002C
:1069B000FFF7AAFF0028E1D1F3E7080001F0EEFF9E
:1069C0000028DAD003780320A342D7D12900300071
:1069D00004F04AFED2E7C046FEFF00008064FF1FBD
:1069E000FFFF00007D64FF1F7C64FF1FF7B50400FC
:1069F000808801F0D3FF0025A84203D00578A08845
:106A000002F008F81C4E3378002B1FD0AB421DD18A
:106A10001A4B28001978FFF777FF002818D00023B9
:106A20003370A3790820A778A688019304F0A4FE08
:106A3000011E0DD0D0230370CA3B8370019B4770A9
:106A400086808371280004F0AFFF01E0002DE8D1BB
:106A5000A0880B4B8200D358002B01D0FFF762FFB8
:106A60001721A088FFF768FDA08801F027FDA08806
:106A700001F0FEFDF7BDC0467D64FF1F7C64FF1F73
:106A80008464FF1FF0B587B01D000CAB1B880700A6
:106A900001930DAB1B88142002930EAB1B881600CC
:106AA00003930FAB1B880091049310AB1B880593D5
:106AB00004F062FE041E1AD0D0230370CB3B477053
:106AC0008370C670062229000430002D11D004F016
:106AD00093FF019B21006381029B0098A381039B8C
:106AE000E381049B2382059BA37404F05DFF07B040
:106AF000F0BD04F071FFECE7F7B5009308AB1B881D
:106B000007000C200D001600019304F035FE041E52
:106B100013D0280001F042FF00280FD00078D023C6
:106B20002370C93BA370009B21002381019B6770E8
:106B3000A580E680638104F037FFF7BD014B18782C
:106B4000EDE7C0460843FF1F13B5040064890389BD
:106B5000C2888188C0780094FFF7CEFF13BD000083
:106B600010B5044C2068002803D004F0A5FD0023D4
:106B7000236010BD8864FF1FA122F0B581889200B8
:106B80004A43384B384F1B6804009B189D229200E3
:106B90009B18827989B01A603B68002B5FD01D7802
:106BA000324B1B68002B04D05B68002B01D0002007
:106BB0009847260008363100E079FFF7B7FD237DBE
:106BC000E0710200E0780493638A29000393238A2A
:106BD0000293E3890193A38800933300FFF752FFE8
:106BE000E378002B0BD1E289A379A1880292019668
:106BF000E27928000092012201F0DAFEE0703B68A1
:106C0000002B20D0FFF7ACFF194D287800281AD0B0
:106C1000184B1978FFF778FE002814D02B78E67807
:106C200008200793A78804F0A7FD011E09D0D023F0
:106C30000370CA3B4670837087808671079804F0A2
:106C4000B3FE00232B701721A088FFF775FCA088E6
:106C500001F034FCA08801F00BFD09B0F0BD064B3B
:106C60009DE7C0463409FF1F8864FF1F9C64FF1F17
:106C70007D64FF1F7C64FF1F0843FF1FF8B50700FA
:106C800008000E0001F08AFE041E18D02620FFF72F
:106C90008DFC051E00D12578062004F06DFD041E34
:106CA0000DD00021062204F097FED0232370C23BB2
:106CB00021006770A370A680E8B204F075FEF8BDED
:106CC000F0B585B001930AAB1B78070002930BABBC
:106CD0001B7808000D000092039301F05FFE061E72
:106CE00022D0102004F048FD041E1DD010220021E7
:106CF00004F072FE2620FFF759FC002800D13078FE
:106D0000D0232370C13BA370009B21002372019B01
:106D100067706372029BA580A372039BC0B2E3728B
:106D20000C9BE36004F040FE05B0F0BDF7B50D002C
:106D3000019001F033FE071E20D00E2004F01CFD50
:106D4000041E1BD02620FFF731FC061E00D13E7822
:106D5000D0232380C53B0622A370F91DE01C04F05C
:106D60004BFE019B2A0063810123DD401A401D4038
:106D7000210022736573F0B204F016FEF7BD000027
:106D8000F0B585B0029010000D0017000A9E039325
:106D900001F004FE041E31D0029B002B2ED1039B78
:106DA00002795B0724D5122313430422002E08D155
:106DB0000B99002905D10C99002902D10D990029C0
:106DC0001AD01A430D9B2271002B00D0C9E0002E6F
:106DD00000D1CFE0002D00D0CCE0606A002801D0C7
:106DE00004F06AFC1C21300004F056FD606205E0EE
:106DF00002239A430E33D7E793432371654BBA00BE
:106E0000D458002C00D1AAE0002E10D0236A002B09
:106E100003D11C2004F058FC20625E4BBA00D3580A
:106E2000186A002803D01C22310004F0E5FD0C9BF9
:106E3000002B12D0574CBB001D596B6A002B03D19D
:106E4000162004F041FC6862BB00E358586A002831
:106E500003D016220C9904F0CFFD0D9B002B11D00E
:106E60004C4DBC006659B36A002B03D1142004F0CA
:106E70002BFCB0622B59986A002803D014220D997C
:106E800004F0BAFD380001F089FD051E67D0414BC2
:106E9000BA00D358002B62D01A6A3420002A00D1DD
:106EA0001C389A6A002A01D0143080B20B9A002A4A
:106EB00001D01C3080B25B6A002B01D0163080B24A
:106EC00004F05AFC041E4AD01822002104F084FD6C
:106ED0002620FFF76BFB0190002801D12B7801934E
:106EE000D0232370029B200063700A23294EA370D5
:106EF000039BBD00A371AB59A780196A1830002904
:106F000005D01C22A06004F077FD200034307359B6
:106F1000996A002907D0030014221433E060029319
:106F200004F06AFD02980B9B002B08D003001C2282
:106F30001C330B992061029304F05EFD0298735993
:106F4000596A002903D01622606104F055FD6B4692
:106F50002100187904F028FD3800FFF7E3FC05B0A4
:106F6000F0BD10220D9B0D991B69A018236204F03F
:106F700043FD2CE70B9B002B00D13FE7012D00D0F8
:106F80003CE7606A002801D004F096FB1C210B98B6
:106F90002AE7C0468464FF1F10B5044C206800280F
:106FA00003D004F089FB0023236010BD7864FF1F29
:106FB0000B4B07B51A68002A01D100200EBD6946A7
:106FC000531C012012780731FFF772FC0028F4D01F
:106FD00002780123100018401A42EED0EEE7C046B6
:106FE0009464FF1FF0B51F4F01203B6887B0002B52
:106FF00025D09B78059300F0B3FB002821D00A2010
:10700000FFF7D4FA04000B20FFF7D0FA164B050067
:107010001E78731E9E413B68F6B2191DD878FFF7A3
:1070200057FB3B682900DA7A043303929A7901937B
:107030000292009033002000059A04F0BDFD07B0D5
:10704000F0BDFFF7B5FF002805D00620FFF7AEFA28
:1070500004000720D8E70820FFF7A8FA0400092059
:10706000D2E7C0467864FF1F7464FF1F70B50A4EF4
:10707000040033780D00FF2B0DD0042004F07CFBBE
:10708000011E08D0D0230370CE3B45708370C470BE
:10709000307804F089FC70BD1843FF1F70B5040000
:1070A00006200D0004F068FB011E0AD0D0230370F7
:1070B000CD3B8370054B44701B688580187804F0C5
:1070C00073FC002C01D0FFF767FF70BD7864FF1FD1
:1070D000F8B5264F06003B680D001124002B05D1A2
:1070E0000522234B1B78134202D112242000F8BD45
:1070F000204A10241268002AF8D01278002AF5D00D
:10710000DB0719D52B789A1E012A1AD80C2004F017
:10711000DBFA132438600028E8D000230A224370E9
:1071200029000670023004F067FCFFF75BFF041EC5
:107130000AD0FFF731FFD9E700F012FB0028E1D1B8
:10714000E4E7002BE2D0D0E70B4B1B78032BCDD12B
:107150001D20FFF72BFA094B18800028C6D0084BDA
:1071600004211878074A04F0D7FCBFE77864FF1FB2
:107170007564FF1F9464FF1F7464FF1F7264FF1F18
:10718000A064FF1F60EA0000F7B50193194B1400DB
:107190001A78052306000F0012201A4221D0012977
:1071A00020D1154B1D68002D1BD002201F2C18D894
:1071B000002C02D0019B002B13D0104B1F221E70FD
:1071C0006E1C0021300004F007FC01992200300001
:1071D00004F012FC310020002C70002F06D004F0C7
:1071E0009BFBFEBD064B12201D68DCE704F014FA81
:1071F000F7E7C0467564FF1F9464FF1F1843FF1F25
:107200009064FF1FF8B50F4E12243368002B17D07F
:107210001B780F3C834213D100250B4F0221387895
:1072200004F022FB094B042138781D8004F01CFB7C
:10723000074B28001D8033685C7004F0EDFB0400F0
:107240002000F8BD7864FF1FA064FF1F8C64FF1F3F
:107250007264FF1F70B5012823D11B4C2388002BBB
:1072600003D01A4A1578002D07D0194B1B68002B44
:1072700002D01878FFF7C6FF70BD3B2B02D93C3B0C
:107280002380F9E7134E0221307804F0EDFAFA2258
:107290002388920002215A43307804F03DFA258079
:1072A000EAE70B4B1B68002BE6D00B4B1B785B0708
:1072B000E2D5084B0221187804F0D6FA0022024BDE
:1072C0001A80FFF769FED7E78C64FF1F7064FF1F09
:1072D0007864FF1FA064FF1F7564FF1FF8B51E4D83
:1072E0002868002803D004F0E7F900232B601B4E28
:1072F0003068002803D004F0DFF900233360184F12
:1073000005243B7818002040234221D0154800F086
:107310002BFA3B78234213D0202004F0D5F92860C3
:10732000002813D02022002104F056FB202004F076
:10733000CBF9041E306005D02022002104F04CFB64
:10734000002004E0286804F0B7F92C601320F8BD91
:1073500000F00AFAF4E7C0469464FF1F9064FF1F30
:107360007564FF1F0C43FF1F10B50A4C23681A1EDB
:107370000ED0002808D10130587004F04DFB0028D1
:1073800005D02368002B02D00021FFF787FE0122E1
:10739000100010BD7864FF1FF7B5274E0500336855
:1073A0000191181E21D05C78244F012C30D1FFF7B9
:1073B000FFFD002825D02000FFF7F8F80400412841
:1073C00014D91F4B022118781E4A04F0A5FB1E4B4E
:1073D0003C3C1C80022233685A703B78002B14D14D
:1073E00028000199FFF75AFE0120FEBDFA22920003
:1073F0004243002AEED0124B0221187804F08CF997
:10740000E8E7FFF7D3F80200F3E700233B70EBE770
:107410003B78002BE8D1032004F0AEF9011E08D020
:10742000D0230370CC3B457083703368187804F028
:10743000BBFAFFF7B1FDD7E77864FF1F7064FF1F49
:10744000A064FF1F60EA00008C64FF1F10B517499D
:10745000838802008B4220D011D815498B4217D067
:10746000144900205B1899B2012907D89268117855
:107470005A425341D8B2FFF7F9FD012010BD0E4A20
:1074800000209B1807229BB29A424041C0B2F5E708
:1074900083681878FFF768FFF0E7836899785A786F
:1074A000090218781143FFF777FFE7E70A20000089
:1074B00006200000F8DFFFFFAFDFFFFF014B187071
:1074C0007047C0461943FF1F10B5064C207001F0ED
:1074D00041FA207804F070FA0521207800F062FD6E
:1074E00010BDC046A064FF1F0BB273B50D00002B8A
:1074F00000DBC4E0884B187804F086F9041E0ED037
:107500000378912B0FD0A22B00D1A1E0834B1878E8
:10751000FF2852D0210004F047FA00284DD18020E6
:107520000002684076BD43780F2B76D013D8052B28
:1075300070D00E2BEAD18088794B98422BD8794BAA
:1075400098421BD8784B9842E0D1A3681878591C10
:10755000FFF774F838E03E2BD8D18378032B74D032
:107560006CD8012B6ED0022BD0D1704B1B68002B36
:1075700023D05B68002B20D098471EE06C4BC018CE
:107580000C28C3D804F0A8FA1DC2C2150BC20B0BFD
:107590000B3223C23C00674BC0180728B6D8664B95
:1075A0001B68002B09D01B68002B06D020009847D1
:1075B0000AE0A3681878FFF7C7F8200004F064F821
:1075C000ADE7A068FFF762F800289FD0F5E7A36851
:1075D0001B78002BF1D0554B1B68002BEDD01B689E
:1075E000002BEAD0210055489847EDE74F4B1B6828
:1075F000002BE2D01B68002BDFD021005048F3E7BE
:10760000504B1B68002BD8D05B68002BD5D02100D5
:107610004348E9E7FFF7EAF9CFE780884A4B984209
:1076200003D04A4B984200D070E7464B1B68002BB2
:10763000C3D05B68002BC0D02100D5E7153B012BE0
:10764000BBD963E7FFF798FAB7E7FFF77DFAB4E72E
:107650003F4B1B78042B07D100236A461380017926
:10766000408800F0C5FCA8E7364B1B68002BA4D06F
:107670005B68002BA1D00100364898479DE70124A4
:1076800021420AD0294B1B68002B04D05B68002BD9
:1076900001D000209847012043E78B070AD5264BED
:1076A0001B68002B04D05B68002B01D0200098479A
:1076B000022036E70421280008400D4200D131E7BE
:1076C000254E3388002B21D0013B9BB23380002B09
:1076D0001AD1FFF7DBF800280AD0204B1C70164B9C
:1076E0001B68002B04D05B68002B01D0200098475A
:1076F000FFF7C6F8694601F001FD6846FEF7FEFF98
:107700001D20FEF753FF308004200AE7024B187853
:1077100004F0AAF8F8E7C046A064FF1F1943FF1F52
:107720000E20000001200000091000009864FF1FD7
:10773000FEDFFFFFAFDFFFFF9C64FF1F0C20000098
:107740000B2000008064FF1F0D20000013200000AC
:107750007564FF1FFFFF00007264FF1F7064FF1F4E
:1077600010B501F09BF910BD014B18607047C04681
:107770009C64FF1F0B880020162B01D817230420C0
:10778000014A13807047C0464A64FF1F00207047BB
:10779000074A03001188814207D09188002099424E
:1077A00002D101308000101870470020FAE7C0466F
:1077B000A864FF1FF0B58F7806000D00C5B01E2F1E
:1077C00015D1FFF7E5FF051E03D10024200045B0C9
:1077D000F0BD00223B003100C078009200F0B2FB07
:1077E0000400A81C00F0D2FBFF23EB70EEE7264B51
:1077F000062403931B78FF2BE8D0182FE6D87B08CC
:10780000224A013BDB0002929A589446002ADDD0BE
:10781000029AD3185B68002BD8D00878002802D1D0
:107820004B78012B02D10624122FCFD107AFAB88A2
:10783000697800976446AA68A047041EC6D1AB7851
:10784000029A5B08013BDB00D318390030005B680B
:107850009847041E0BD1AB78042BB6D0039A3100A5
:1078600010782200009700F06DFB0400AEE76A7804
:10787000002AABD1AA7805A93B88087130000A70AC
:107880004B80FEF747FBA0E71C43FF1F2CBE0011F7
:107890001D4B37B5050098420BD000290AD1FFF7E0
:1078A00077FF002805D11948FFF772FF002800D0A4
:1078B000058037BD01291AD1FFF76AFF041EF8D0F1
:1078C00001235B420380A378FF2BF2D0FE2B07D06D
:1078D0000023E0781422009329001E3300F032FBCD
:1078E000A01C00F053FB01235B426380E1E7022907
:1078F000DFD1013901F0BEF80028DAD12800FFF706
:1079000047FF041EDFD1D4E7FEFF0000FFFF0000A9
:10791000022210B5074B52421A80074801325A80A2
:107920009A80DA8000F07EFA044801F025F8002001
:1079300010BDC046A864FF1FB577001191780011F3
:107940000388F7B50400002B02D102252800FEBDF4
:1079500042680221137825485268FEF7A5FD0028E9
:107960002ED0234F01253A88002AEFD0802321888A
:107970005B0201259B1A9942E8DC0C2003F0A4FE6F
:10798000061E31D03B8822889C46002318000195B2
:1079900061469DB2491989B2AA421BD8002801D07C
:1079A00062443A8000233000082208C0210004F01D
:1079B00023F8104A1368002B13D100251660C5E781
:1079C0006268022113780C485268FEF76DFD0028AA
:1079D000C7D1BAE760681D014019418101330198A0
:1079E000D6E71A001B68E6E71325AFE79ABE001139
:1079F0001A43FF1FA464FF1F98BE0011014B1870AB
:107A00007047C0461C43FF1F14230A0010B51A40DC
:107A1000194204D00122102101F048F810BD4B0694
:107A2000F9D4012088434000F8E710B514008B0614
:107A300004D50122102101F039F810BD08230A00F5
:107A40001A40194202D14BB2002B0FDA102101F07B
:107A50002DF8002808D02300F2331B78002BECD03F
:107A6000F1342378012BE8D10020E6E703208907D1
:107A7000FAD4E2E7F0B51F00184B85B01C680190FE
:107A800002910392002C27D1200005B0F0BDA5681B
:107A90003301ED186B89019A934211D3029A9342F4
:107AA0000ED8002F04D10A9B002B10D12C00EBE73D
:107AB0003B002978039A6868FEF7F6FC0028F2D1AB
:107AC0000136B6B2A388B342E1D82468DAE7A368E6
:107AD0000A9A5B891380E9E70026F3E7A464FF1F95
:107AE00037B50C000A8849880123914217D3002A30
:107AF00015D0651D23792A0002210A48FEF7D4FC1F
:107B0000102300280BD023796188208800242A00C4
:107B10000094FFF7AFFF0A23A04200D02300180013
:107B20003EBDC0469ABE001113B50A0008884988B8
:107B3000012388420BD8002809D00024137905328C
:107B40000094FFF797FF0A23A04200D023001800FB
:107B500016BD13B50A0008884988012388420BD84E
:107B6000002809D00024137905320094FFF782FF22
:107B70000A23A04200D02300180016BDF0B58BB038
:107B800003904A8808880E000123824255D30028BA
:107B900053D00023012704AC237000227188130006
:107BA0000092FFF767FF051E3ED02078002835D1F0
:107BB0002B78022B18D167706A8983000130E31893
:107BC00080005A8069680222201803F015FF23788C
:107BD0000133DBB22370042B19D93B0068890130D3
:107BE00080B2002BD9D01FE00223637012235843C8
:107BF0006A89231804305A8069681022201803F01B
:107C0000FBFE23780133DBB22370002BE5D10C4A55
:107C10006B899B185A425341DBB2DFE76378012B33
:107C2000E4D12B78022BC7D022780A23002A04D073
:107C300021000398FEF798F9002318000BB0F0BD5F
:107C40000100FFFF0F4BF0B504001868002816D0A4
:107C500083685D89A54207D88288AE18B44203DAEA
:107C600012019A18934201D10068EFE71E005F8964
:107C70001036A74204D1002900D00D801800F0BDB5
:107C80003300EFE7A464FF1F70B505000C000888FF
:107C90000021FFF7D7FF03000120002B04D02200B2
:107CA0002800197AFFF7C1FE70BDF7B50C0000255A
:107CB00001902300EE331B78AB4201D800200AE08C
:107CC0006B00E65A00213000E718FFF7BBFF0028E1
:107CD00002D126800130FEBD017A0198FFF794FEA3
:107CE000002802D03B882380F5E70135EDB2E0E7BC
:107CF00010B5040008880021FFF7A4FF030001204D
:107D0000002B03D02000197AFFF77EFE10BD000083
:107D1000054B1B68002B01D1180004E09A685289BA
:107D20008242F6D198887047A464FF1FF0B50E27F1
:107D3000002687B0039302ABFF183E8005001F4B5F
:107D400040891400984207D02B78013000976A6868
:107D500080B2FFF78FFE060002212B7818486A6870
:107D6000FEF7A2FB00280FD06C892000FFF7D0FFA0
:107D7000002802D0013C0419A4B2039B002B00D0C0
:107D80001C80300007B0F0BD02212B780D486A68D6
:107D9000FEF78AFB0028E7D102212B780A486A689F
:107DA000FEF782FB002807D0002EDED03B88A342DE
:107DB000DBD17489013CDFE76C89DEE7FFFF00005F
:107DC0009ABE001198BE001196BE001110B50C00AD
:107DD000FFF7DEFC03000220002B0AD0002C00D0AD
:107DE00023609B781720FE2B03D00138FF2B00D196
:107DF000002010BD73B50D0001A904001600FFF7A7
:107E0000E5FF172805D0002E04D129002000FEF739
:107E100027F976BD01221021200000F047FE00283E
:107E2000F3D0F6E7014B18607047C046B464FF1FFB
:107E300037B56B469D1D010004000222280003F0A7
:107E4000C3FC2B88B02B0ED12379122B09D1230030
:107E5000FA331B78012B06D10121608800F0E0F88D
:107E600001E01B2BF8D037BD10B5054B042118706D
:107E700000F098F8FFF74CFDFEF770FB10BDC04610
:107E8000B864FF1F0020F0B50BB20F0087B083422B
:107E900034DA274B187803F0B7FC051E2BD0037893
:107EA000A02B25D103AE3100FEF7E4F8041E0BD160
:107EB000B378DB0724D51F4B06341B68002B03D097
:107EC0003100688898470400A868002801D003F0B2
:107ED00033FC002C08D1184A039B1340174A9342E5
:107EE00006D0B3781B2B03D00121688800F098F8E6
:107EF000280003F0C9FB80200002784007B0F0BDE5
:107F00000F4B1B68002B10D0310068889847041E67
:107F1000DAD07378002BD7D1B27801A90A704B80E0
:107F20000C716888FDF7F6FFCEE70624F1E7C0463E
:107F3000B864FF1FB064FF1F00FFFF0000011200C4
:107F4000B464FF1FF7B50190FC200D0017001E0060
:107F500003F012FC04001320002C12D0B0232000E8
:107F60002370089BF4226770658026710830002B0F
:107F700008D0190003F040FD2100019803F014FD22
:107F80000020FEBD089903F027FDF5E710B5041E9B
:107F900006D00078FD2803D803F076FCFF23237079
:107FA00010BD00000A1F93B210B504000220032B7D
:107FB00005D882400020024BD1529B189C7010BD06
:107FC000D864FF1F0B8870B5043B04000D0002202D
:107FD000032B0BD80121200000F04CFD03001420DE
:107FE000002B03D02900200000F0DEFB70BD000054
:107FF00007B51300034A00920A00012100F02CFC8F
:108000000EBDC0462D82001107B5019203220092D9
:10801000024B0A00122100F049FC0EBDAB82001198
:1080200007B56B4601AA11800449D8800878063349
:10803000012802D1190003F077FC07BDB964FF1FC6
:108040000C4B10B518700023FF210B4A13801381CD
:1080500093819380094A5380137051729381937274
:10806000D174D3821375517703F08EFD00F0FCF9C3
:1080700010BDC046E864FF1FD864FF1FBA64FF1F2D
:10808000F0B58DB06B46002003910C229B5E8342BD
:1080900000DBB0E05D4B187803F0B6FB051E00D1A5
:1080A000A4E00378902B00D09DE006AF0100468845
:1080B000380000F013FA79680400002900D19CE030
:1080C0003B88052B6ED13B89032B1CD905AC2000C6
:1080D00000F0A2F86288172A61D83989131D9942E5
:1080E00031D17968237804310291D90738D5607885
:1080F00000F08EF9071E06D0002303712378012BB0
:1081000008D0132B23D0A868002800D178E003F012
:1081100013FB75E06288029909A800F0A6F80290A6
:10812000380000F08BF909AA2378387A01920022EE
:1081300031000092029A00F012F9380000F064F960
:10814000029B002BDFD0300000F080F9DBE70378E2
:10815000032BD8D16288029909A800F0D6F8DEE78F
:10816000122B13D1029909A800F0B5F8021EEAD12A
:1081700027498B88002BC6D0887909A923780191DB
:1081800061780091310000F0EAF8BCE7002302AA10
:1081900093833000617809AAFFF72AFFB3E71D4BEC
:1081A0000993F6E7042B02D09A1F012AABD8184A8C
:1081B000043B9B00995A0029A5D0D2189078310031
:1081C0003A0000F0AEF800289DD13B88042B03D084
:1081D00001213000FFF724FF012C04D1A8680028FA
:1081E00001D003F0A9FA280003F04EFA8020039B87
:1081F0000002434018000DB0F0BD012800D182E715
:1082000001213000FFF70CFFEDE7C046E864FF1FD7
:10821000D864FF1F010017000B7803704B78437080
:10822000CB788A781B021343438070470A88030087
:1082300002700A88120A42700A88012A06D14A8806
:1082400082704A88120AC27004207047022082425B
:10825000FBD14A8804309A704A88120ADA708A88F8
:108260001A718A88120A5A71EFE710B504000120CA
:1082700082420CD94B780A781B0213432380834235
:1082800006D1CB788A781B0213436380002010BD8F
:10829000022BFBD1CB788A781B02134363804B7986
:1082A0000A791B021343A380F0E70B8803700B8845
:1082B0001B0A43704B8883704B881B0AC3708B88E2
:1082C00003718B881B0A4371CB888371CB881B0A8F
:1082D000C3710820704703000120082A14D14A788E
:1082E0000878120202431A80CA7888781202024380
:1082F0005A804A790879120202439A80CA798879A9
:10830000120202430020DA80704710B504000120F9
:10831000022A05D100204B780A781B0213432380E0
:1083200010BDF8B5060010200F00150003F024FA68
:1083300004000120002C0ED0A0230C222900238051
:108340006780201D002D07D003F056FB2100300070
:1083500003F02AFB0020F8BD03F03EFBF6E7F7B57B
:108360001E00009008AB142017001D78019103F047
:1083700003FA041E12D0A2230370019B47704380AE
:10838000099B057146710C220830002B07D019009B
:1083900003F032FB2100009803F006FBF7BD0999BA
:1083A00003F01AFBF6E737B5041E0FD04388002B05
:1083B0000CD00025C1881323007A1722019500955F
:1083C000FFF7CDFFFF2365806372257037BD000086
:1083D00010B50C4904004A88002A09D08B89002B6B
:1083E00005D00020CB8A0222834201D010BD012299
:1083F00013000A20434300204032C854C81842806A
:108400000472F3E7BA64FF1F0023438003707047D0
:10841000094B00211A0010B55C88002C06D01C798D
:10842000844203D10A234B43D01810BD01310A33D3
:108430000329F1D10020F8E7BA64FF1F10B504004A
:10844000407A03F021FAFF23637210BD70470430B5
:1084500010B580B203F048FB002803D00421494244
:1084600003F0BAF910BD000070B50025104CA068EB
:108470002580A581A580A84202D003F05DF9A56002
:1084800000250C4C0C4B606D1D80230058331D7073
:10849000A84202D003F050F9656500256068002805
:1084A00001D003F049F9013508340A2DF6D170BD29
:1084B0008065FF1F2465FF1F7465FF1F70B5041ED4
:1084C00009D1054D2880A881A880A868002802D07D
:1084D00003F032F9AC6070BD8065FF1FF0B54B88CA
:1084E00085B00193002343600A7905000F00022A3A
:1084F00000D07BE0CA88032A17D98B685E78197888
:108500003602DC78D8790E4399781B7A24021B0254
:108510000C43034353495BBA0B80331D93421ED176
:10852000042C04D0631F022B0ED9012015E0019A00
:108530004D4B1201D35A002B06D00198FFF7BEFF16
:108540004A4A1369013313610421B8682E812C80D3
:10855000494203F041F96860002005B0F0BD434D89
:10856000042C06D0631F022B0FD9EB680133EB609C
:10857000DBE7019A3C4B1201D35A002B05D001983E
:10858000FFF79CFF2B6901332B61374B30000293BF
:10859000019B029A1B010193002301998C468B5287
:1085A000130063449C8003939E81FFF750FF039B5D
:1085B000041E986016D00421B868494203F00CF9F3
:1085C000FA880100043A200003F016FA0199029A91
:1085D000FB888A5A043B9B18029A8B522B68013302
:1085E0002B60A2E7AB690133AB619EE71E4B0293A0
:1085F000019B1E01029BF35A002B2DD002998C196E
:10860000A068002828D0012A26D1FA889B189BB29E
:108610007352A189994217D39B1AC018B96803F005
:10862000EBF9029BA289F35A934200D07DE7002226
:108630002B81A3882B80A3686B60029BF2520B4AAC
:1086400053680133536070E7084A936801339360BD
:108650000198FFF733FF68E7044A53690133536118
:10866000F6E7C046EA64FF1F8065FF1FF064FF1F46
:1086700070B5051E15D10B4C0B4B188023005833D9
:108680001870606D002802D003F056F8656525006B
:1086900050356068002801D003F04EF80834AC4231
:1086A000F7D170BD2465FF1F7465FF1FF0B517007B
:1086B000A12285B0920001934243394B06001B680A
:1086C0000C009B18D933FF331D78FDF741FF0430B0
:1086D000854204DD3000FDF73BFF0430C5B2BD42EA
:1086E00007D33A0000213000019B03F03DF905B0AB
:1086F000F0BD2900380003F04FF82300C6B2503314
:108700001E700393019B29006365380003F09CF8F9
:10871000CBB20293002B02D0039B01361E700026C1
:108720002300503303931B78B34204D8606D0028B4
:1087300031D10020DBE7029A2800002A04D0013B57
:108740001000B34200D02800F700E719387003F09A
:1087500063FA786000280ED03A78019903F04CF95A
:10876000019A3B780136D3180E4A0193D369F6B2C9
:108770000133D361D4E7039B18706065A74205D12C
:10878000084A1320D36A0133D362B0E7606802F06D
:10879000D3FF0834F2E702F0CFFF00236365C8E798
:1087A0003409FF1FF064FF1FF7B50D000700042117
:1087B000686803F011F82B89040003702B891B0AE9
:1087C00043702B8883702B881B0AC3702E89022567
:1087D0000436F6B2F42E15D81B4B9F4214D10C2050
:1087E00002F0CAFF1135011E0CD0902303708E3B9E
:1087F0000371043B4380154B8460C680187803F0F6
:10880000D3F800252800FEBD5C237B43104AD31813
:108810000093583301931B78002B0FD103003200D3
:1088200038000099FFF742FF019B05001B78002BE1
:10883000E8D13800009903F067F8E3E7054A072517
:10884000536A01335362DDE7FEFF0000E864FF1F57
:108850002465FF1FF064FF1FF0B587B0009017205C
:108860000F0016000193FFF7F2FD1325041E19D027
:108870000C98031E02D00199201D9847030AE3704B
:10888000052302AAA07004309081277000986670BA
:1088900003A993800494FFF787FF051E02D02000F0
:1088A00002F04AFF280007B0F0BD0000F0B587B025
:1088B0001F000CAB1B780391059301210DAB060043
:1088C0001C78049200F0D6F81425002821D020004E
:1088D000FFF77EFD0135041E1BD01149059B0A7868
:1088E00003700132D2B2131EC68001D101231A00D7
:1088F0000B7022713000049B03990097FFF7ACFFC7
:10890000051E09D1230021000648074A093303F058
:108910008BF8280007B0F0BD002363802370F8E7D0
:10892000EC64FF1FA783001130750000F8B5050047
:108930000E00064C064F2368002B02D031002800A1
:1089400098470434BC42F6D1F8BDC0469065FF1F7D
:10895000A465FF1F0123064A5B4253800023137165
:108960005362044A136053609360D360136170478D
:10897000A465FF1F9065FF1F0200002310B5064984
:108980009C000859002801D1625010BD0133052B0D
:10899000F6D11320F9E7C0469065FF1F034A5388BC
:1089A000181A43425841404210407047A465FF1FC7
:1089B000F0B585B002930AAB1F780CAB1B88009012
:1089C00008000E0001920393FFF7E8FF0500112055
:1089D000002D1BD10E48FFF7E1FF04001520002CED
:1089E00014D006220B99A771E01D03F005F8019B36
:1089F00030002371029B29006371009B6680237005
:108A0000039B6562E381FFF791FF280005B0F0BD8D
:108A1000FFFF000010B5FFF7C1FF04000220002C8B
:108A200012D060880121FFF781FF606A002801D021
:108A300002F042FE28220021200002F0CDFF012397
:108A400000205B426380207110BD000030B5074AF2
:108A5000074C5588010013780020A54204D05B1A0A
:108A600059424B415842104030BDC046A465FF1FDB
:108A7000FFFF0000084A10B501230C00904208D007
:108A8000FFF78CFF031E04D0037923405A1E934145
:108A9000DBB2180010BDC046FEFF0000024B187983
:108AA000431E9841C0B27047A465FF1F70B5040013
:108AB0000D001600FFF772FF002804D10D4B9C42F9
:108AC00000D0143070BD416A03790520002907D019
:108AD00012221A40102A02D10520002EF2D10F20B6
:108AE000DB06EFD5897E0C20A942894149424942E3
:108AF0000840E7E7FEFF0000030010B5002800D1A2
:108B000010BD0348034A41889142F9D09847F7E7DE
:108B1000A465FF1FFFFF0000002330B5C45CCD5CDF
:108B20006C40D4540133102BF8D130BD0F230022F8
:108B300010B5C45C64002243CA54C25CD209013B34
:108B4000F7D210BD0200010010B52032103102F042
:108B5000A3FD10BDF0B58BB0039010200593170056
:108B6000049102F0B1FD0090102002F0ADFD009BD9
:108B700013240190002B05D000280CD11324009859
:108B800002F09AFD019B002B02D0180002F094FD28
:108B900020000BB0F0BD102002F096FD0600102062
:108BA00002F092FD13240500002E00D1AEE0002853
:108BB00019D01022002102F00FFF32002900039883
:108BC00002F06AFD041E0ED133787F2B51D830009D
:108BD0000099FFF7ABFF009B1B787F2B53D80199BF
:108BE0000098FFF7A3FF300002F066FD002D02D0D1
:108BF000280002F061FD002CC1D1102002F064FDBC
:108C00000600102002F060FD0290002E7CD00028AB
:108C100078D03A000F3223000125121105D00F330E
:108C20003B4015B25A4253411BB26A1E1201002B3F
:108C300033D0049BD2B298180099029AFFF76CFFC8
:108C4000013D10220021300002F0C6FEADB2049FAB
:108C50002D017D19AF4242D0002C33D0300002F0FC
:108C60002BFD029B002B00D189E7180002F024FDA8
:108C700085E729003000FFF759FF28002549009AB1
:108C8000FFF74AFFA7E729000098FFF74FFF2800EA
:108C90002049019AFFF740FFA5E70F210F400499F3
:108CA0008A18D9B28F4208D9D15C06A81954013369
:108CB000102BF6D1029A0199C0E7791A4842414136
:108CC000C901F2E73900300006AAFFF725FF32009C
:108CD000039806A902F0E0FC10370400BAE7002C64
:108CE000BCD13000029906AAFFF716FF320006A990
:108CF000039802F0D1FC082204003100059802F02C
:108D00007BFEABE71324A9E71324AAE7002800D0D1
:108D10006EE733E7A0BE0011F0B58BB00F00160070
:108D20000225009000283FD0002A3DD00B1DDBB269
:108D30001800029302F0C8FC1135041E34D0FDF770
:108D400047FD05003A000099201D02F0B5FEEBB288
:108D50000393E3702B0CDBB22F0A00936370FFB216
:108D60002B0E2370A7700193FDF72CFD102201003C
:108D700006A802F0A1FE2100029A04AB06A8FFF7A4
:108D8000E9FE051E0DD1039B08223370009B04A948
:108D9000B370019B7770F370301D02F08DFEFDF70C
:108DA0001DFD200002F088FC28000BB0F0BDF0B5DE
:108DB0008FB00D00149E039004920593002A03D1F6
:108DC000022420000FB0F0BD002EF9D00398FFF769
:108DD000E5FD1424071EF4D07278337812021A438A
:108DE000B3781B041343F27812061A43036A019204
:108DF000934201D30133E3D1002D03D03B79012409
:108E00009B07DED50822002106A802F0E5FD059BA0
:108E100013240433DBB21800029302F055FC051E44
:108E2000CFD0059A0499043002F046FE04223100A6
:108E3000280002F041FE3900102210310AA802F089
:108E40003BFE2900029A06AB0AA8FFF783FE041E28
:108E50000FD1082206A908A802F02EFE0822311D13
:108E600008A802F069FE012807D101990398FDF7CF
:108E7000C9FC280002F020FCA3E70124F9E7000068
:108E800070B51C4C05002368181E10D0002D14D19D
:108E90001A78002A0CD1981C083202F0ADFD02F0BD
:108EA00063FE0135002808D123681D70012070BDC4
:108EB0000A331800082202F09FFD2368002BF5D02A
:108EC000122002F059FC061E0DD0C1232168037048
:108ED000457002311022023002F08EFD236831000D
:108EE000587802F061FD206802F0E6FB0023236061
:108EF000DCE7C046CC65FF1FF8B504002020FDF775
:108F000055FB0D4EA700BB590500002B0DD00028C6
:108F10000BD0D878FF2809D108492A000C55F359FD
:108F200007480333611802F07FFDF8BD290002F005
:108F30009BFD0028F0D1F8E7E865FF1FD065FF1F13
:108F400051A1001170B5064D84006359002B05D066
:108F5000D87802F099FCFF226359DA7070BDC046E0
:108F6000E865FF1F70B506008CB00C0015000021ED
:108F70003022684602F030FD31001022684602F0CF
:108F80009BFD1D2021000322684402F095FD6846E8
:108F9000FFF7D8FD2D21040003222800694402F0C8
:108FA0008BFD20000CB070BDF0B50700160097B027
:108FB00001931CAB1D7830221EAB00910AA8002142
:108FC0001C7802F009FD102239000AA802F074FD95
:108FD0001022002102A802F0FFFC0722310002A8A3
:108FE00002F06AFD072202AB9818631E9C410199AA
:108FF00002F062FD02AB9C732B005A1E934102AA41
:10900000D3730021102206A802F0E6FC06221D9967
:1090100007A802F051FD1A2002ABC01806221F99C2
:1090200002F04AFD102200990EA802F045FD102220
:1090300002AB0EA908781C78013A6040D2B20870E1
:1090400001330131002AF5D10AA8FFF77BFD102278
:1090500012A904000EA802F0CFFC102206AB0EA944
:1090600008781D78013A6840D2B2087001330131A6
:10907000002AF5D10AA8FFF765FD044310222098C5
:10908000E4B212A902F018FD200017B0F0BD70B5CF
:109090000E0014008CB00100102268461D0002F082
:1090A0000BFD3100082204A802F006FD2100082271
:1090B00006A802F001FD6846FFF744FD04001022F7
:1090C000280008A902F0F8FC20000CB070BDF8B52B
:1090D00006000D0000243719AC4200D3F8BD02F0A1
:1090E00053FB030A3B70631CDBB201379D4203D97B
:1090F0000234F054E4B2EEE71C00EDE773B506006D
:109100000C000225002819D0002917D0032101A83E
:10911000FFF7DDFF6B469A793F231A400133134373
:109120006A463000937101A92200FFF71BFF051E5C
:1091300004D10322E01C01A902F05EFC280076BDE8
:1091400003785807DA08C00FD20080009B0710434D
:109150009B0F1843C0B2704707230B40C908C900D2
:109160000B4303707047000070B50400FFF7EAFE80
:10917000134DA4006359002B21D0186A002801D098
:1091800002F09AFA2B59986E002801D002F094FA56
:109190002B59D86E002801D002F08EFA2B59186F87
:1091A000002801D002F088FA2B59586F002801D00E
:1091B00002F082FA285902F07FFA00232B5170BD89
:1091C000E865FF1F0E4B8000C35870B50C00002BE4
:1091D0000FD09D68002D0CD02B78201D0B706B7864
:1091E0004B70A97CFFF7B8FF2B7E23726B69E3609D
:1091F00070BD10220021200002F0EEFBF8E7C0460F
:10920000E865FF1F014B18607047C046E465FF1F0B
:10921000074A03008000825810B5002A06D0D08883
:10922000984203D1012901D1FFF79EFF10BDC0462E
:10923000E865FF1FF0B5264E95B087000B93BB592C
:109240000500099112200A92002B31D0D888FFF72F
:10925000A5FB04001420002C2AD0280010A9FFF739
:10926000B1FFBB591E781D6A002E23D00895FDF76B
:10927000EFFA07000020FDF7F1FA0790A379E61D49
:10928000069310AD0CA9089800F0E2FA0EA9280088
:1092900000F0D7FA0B9B0A990493069B0998029356
:1092A000079B0396019300970EAB0CAAFFF77CFE79
:1092B00015B0F0BDFDF7CCFA06903000FDF7CEFA00
:1092C000E31DA779079310AB06000893DAE7C046C1
:1092D000E865FF1F30B50C4C85002A59030085B0A6
:1092E0000120002A0ED018006946FFF76BFF2B59AA
:1092F0001A78D888054B002A00D1054B6A46072109
:1093000000F0D9FB05B030BDE865FF1F43980011A0
:109310005198001130B5094C8500295985B01022AB
:109320006846253102F068FB2A591121044BD08888
:109330006A4600F0C0FB05B030BDC046E865FF1FBF
:10934000ED98001130B5094C8500295985B01022DF
:109350006846353102F050FB2A591121044BD08860
:109360006A4600F0A8FB05B030BDC046E865FF1FA7
:109370002B990011F7B54D4F86001020F4590D00C0
:1093800002F0A2F9F3592062186A132200286CD067
:10939000033A29009C6802F02FFBF3591A780192D6
:1093A000002A58D11E6A227D317B94465140012209
:1093B000019F114201D167461740217D91433943F6
:1093C0002175377B4F40BC4660460027800701D49B
:1093D0004F081740012102208F40227D82433A43EB
:1093E0002275377B5740BC4660460027400701D4B2
:1093F00097080F400420227DBF0082433A43227524
:10940000627D002794466046727B42400A4201D149
:1094100067460F400121627D8A433A436275777B3C
:109420005740BC4660460027800701D457080F40CC
:109430000220627D7F00824317436775767B00229E
:109440007E40760701D4BA080A400426617D920066
:10945000B1430A4362756A78002A08D06278002A0C
:1094600005D005220533DA7700221000FEBD042264
:109470002979114205D1A17C114202D10533033A69
:10948000F1E7019A21782C78002A02D10A00210004
:10949000140018220429E8D8042CE6D805206043DB
:1094A000034A05331218525CDDE7C046E865FF1F2A
:1094B000B0BE001110B50A001121024B00F0FBFAFA
:1094C00010BDC046879900110B0030B587B001ADC3
:1094D0002B806B4604001100981D082202F08CFAC4
:1094E0002A000B212000024B00F0E5FA07B030BD46
:1094F000AF99001110B50A001121024B00F0DBFA00
:1095000010BDC046039A001113B50B0011006A4646
:1095100013706B4604000622581C02F06DFA6A466E
:1095200008212000014B00F0C6FA13BD239A001158
:1095300010B50A001121024B00F0BDFA10BDC04663
:10954000739A00117FB505000B4BAA00D458080090
:10955000002C0FD0666F237FE28821780396266F58
:109560000296E66E0196A46E0094FDF709FC2800B1
:10957000FFF7FAFD7FBDC046E865FF1F10B5172154
:10958000FFF7E0FF10BD000070B50A000D00064BAC
:109590000221040000F08FFA060029782000FFF76E
:1095A000D1FF300070BDC0465399001170B586B030
:1095B00000236A461370836804001D78681E0A2819
:1095C00059D801A902F0F0FA060633373B3F43476A
:1095D0004B4F5300180000F042F9062312284BD0DD
:1095E00000281BD16088FFF7D9F90823002813D081
:1095F0004279002A47D1264B1A78072312070BD548
:10960000244B1A680723002A06D01668002E03D0C0
:10961000290001AAB04703006A4613706B461B7805
:109620006088002B2AD1FFF767FC06B070BD1800D8
:1096300000F06CF9D4E7180000F087F9D0E71800C3
:1096400000F093F9CCE7180000F0ADF9C8E7180076
:1096500000F0C3F9C4E7180000F0F6F9C0E71800FD
:1096600000F0F6F9BCE7180000F013FAB8E71800AC
:1096700000F013FAB4E707236A461370694660885E
:10968000FFF782FFD1E70523012AC5D1024BB8E7D6
:109690007564FF1FE065FF1FE465FF1FF8B52C4FE1
:1096A0008600F35904000D00002B40D0DA88824276
:1096B0003DD15A78062A33D11A78002A2ED00120BB
:1096C00099681A6A097D014206D0157B054203D0CC
:1096D00007225A700120F8BD0220014204D0157BF8
:1096E000054201D00922F4E70420014204D0127B94
:1096F000024201D00B22ECE7164B1B68002BE9D08D
:109700005B68002BE6D020009847BB5900215B78AE
:10971000122BDFD12000FFF715FFDBE70E4BECE744
:10972000112A04D1002900D032252900F2E7002DAA
:1097300008D12000FFF732F9002803D01023027966
:109740001343037121002800FDF798FAC2E7C046D1
:10975000E865FF1FE065FF1FE465FF1F70B50E4E53
:109760008500AB590400002B13D01B78002B11D1BE
:109770000A4B1B68002B04D05B68002B01D0200033
:10978000984773595B78122B03D100212000FFF713
:10979000D9FE70BD024BECE7E865FF1FE465FF1FD3
:1097A000E065FF1F094B8000C3581020002B0CD030
:1097B0001A6A002A09D09B68002B06D0127A1B7EF9
:1097C000101C9A4200D9181CC0B27047E865FF1FF0
:1097D00070B503000D0014000220002A30D00029CB
:1097E0002ED013700B78081D53704B789370FFF7D1
:1097F000A7FCE070012002212B7A23716B7B0340D0
:1098000063716A7B0A401343042263716E7B1640C6
:10981000334363716E7BF608F600334363712B7B31
:109820000340A371287B014000200B43A371297BD7
:109830000A401343A3712A7BD208D2001343A371B9
:1098400070BD10B50A0001000120FFF7C1FF10BD77
:1098500010B50A0001000220FFF7BAFF10BD70B575
:1098600006000C000220002E30D000292ED0737884
:10987000201D0B70B3784B70F178FFF76DFC01225F
:109880003579257271794B100800134093401040D0
:109890000343881010408000C9080343C9000B43EC
:1098A0006373B1794B100800134093401040034399
:1098B000881002409200C9081343C9000B432120BD
:1098C0002373FCF773FE854201D2122070BD222063
:1098D000257AFCF76BFE8542F7D823781820042BF5
:1098E000F4D86378012BF1D80020EFE7030010B51E
:1098F0000220002909D0002B07D00322481C0A703F
:1099000019000D3202F078F8002010BD0300022289
:10991000080010B5002B06D0002904D00E32591CC7
:1099200002F06AF80022100010BD030010B50220FA
:10993000002909D0002B07D00422481C0A70190006
:109940000C3202F059F8002010BD10B5FFF7DEFF11
:1099500010BD03000220002906D0002B04D00522F0
:1099600000200A701B784B70704703000220002B08
:1099700008D0002906D05B7800200B70013B082B33
:1099800000D918307047030010B50220002909D013
:10999000002B07D00622481C0A7019000A3202F078
:1099A0002BF8002010BD10B5FFF7B0FF10BD02006E
:1099B0000B00022010B500290ED0002A0CD0072180
:1099C0001970118859701188090A997011180822A4
:1099D000D81C02F011F8002010BD03000A0002207C
:1099E00010B5002B0CD000290AD0997858780902BC
:1099F00001431180901CD91C082201F0FDFF0020BA
:109A000010BD030010B50220002909D0002B07D09B
:109A10000822481C0A701900921801F0EDFF00207E
:109A200010BD02000B00022010B500290BD0002A47
:109A300009D009211970117818185970511C062283
:109A400001F0DAFF002010BD10B5FFF75FFF10BD79
:109A500002000B00022010B5002A09D0002907D00F
:109A60005178197011180622581C01F0C5FF00200A
:109A700010BD030010B50220002909D0002B07D02B
:109A80000A22481C0A701900063201F0B5FF0020B6
:109A900010BD10B5FFF73AFF10BD02000B00022009
:109AA00010B5002A06D0002904D018005178FFF71D
:109AB00053FB002010BDF0B585B017001E006A46AC
:109AC00006230500080091819380FEF7C0FC132453
:109AD000011E02900CD03800B047041E05D12800AA
:109AE00001A9FEF76FFA041E02D0029801F024FECD
:109AF0002800FFF701FA200005B0F0BDF0B5040022
:109B00008BB0019115000021102202A801F064FF22
:109B1000334EA700B85900283CD0C388A34239D19E
:109B20000378002B36D14278062A18D102000100B2
:109B3000553235310C3006ABFFF7A9FA002829D190
:109B40002000FFF72FFE020006A902A801F054FF33
:109B5000200002A901F0E8FD01200BB0F0BD816EEC
:109B6000002917D00B8A112A28D19D420ED10198C5
:109B70001231093A01F0E0FF012807D1BB5920005A
:109B80009D6EFFF70FFE29000200DEE73221200064
:109B9000FFF7D8FC2000FEF701FF061E1BD0416A2C
:109BA000002918D00B8AAB4215D108220198123136
:109BB00001F0C2FF01280ED1716A0AE09D42E9D18D
:109BC00008220198123101F0B7FF0128E2D1BB59F8
:109BD000996E8A7EB9E7200001F04EFDBCE7C046D1
:109BE000E865FF1FF0B56B4D87007E5985B033786F
:109BF00002900393002B00D087E0B368346A01938E
:109C00007078062817D101221B7D134202D0217BD8
:109C1000114218D10222134202D0217B114251D1AC
:109C20000422134203D0237B134200D08BE0019B1C
:109C30005A7DEB5991E007380428F8D801F0B4FFB9
:109C4000032E42678300B36E002B03D11C2001F06A
:109C50003BFDB066EB599C6E002C1CD010220021FD
:109C6000200001F0B9FE0298FFF79CFD01002000E2
:109C7000FFF72DFA01F088FD208220000821123024
:109C8000FFF725FA0298FFF78DFDA076EB5921002A
:109C9000D888FFF70FFC0822EB591CE0B36E002BAD
:109CA00005D01A00198AF0881232FFF70DFC022243
:109CB000019B197DEB5911423DD0207B10423AD0D7
:109CC000073208E0F488FCF7DBFD01002000FFF715
:109CD00011FC0A22EB595A70029B9C002A595378B6
:109CE000073B042B11D8D088FEF758FE00284ED031
:109CF000C3895A08D2182849029B0298CB542B5981
:109D000041180433254801F08FFE05B0F0BDFCF783
:109D10009FFD03000120834201D100200393EB59F2
:109D2000DE88FCF79BFD039902003000FFF7ECFB97
:109D3000019AEB59117D042211420CD0217B114272
:109D400009D00B22C7E7F688FCF73CFD0100300084
:109D5000FFF7EEFB6BE7019A527D01210A4204D026
:109D6000607B084201D00C22B5E702210A4204D0F0
:109D7000607B084201D00E22ADE704210A4204D0E4
:109D8000627B0A4201D01022A5E71222A3E7FA2241
:109D90005200B0E7E865FF1FEC65FF1F5BA10011F3
:109DA00010B5064B1A780423100018401A4200D050
:109DB0000348FFF727FA002010BDC0467564FF1F57
:109DC0002043FF1F70B50400FFF7D4FA051E43D1EE
:109DD0002000FFF77FFA234EA400A0598268937CED
:109DE000DB0708D50321036A1B790B40012B02D145
:109DF000017F0B430377431DD97F8B1E022B0DD8A8
:109E0000022900D00121C088FCF790FF04213359BA
:109E10001A7F59700A431A77280070BD01290CD1A6
:109E200002231022437000210C3001F0D5FD30597F
:109E300010213530FFF74BF9EEE70529ECD102236D
:109E4000D118437010220C3001F0D6FD0423325992
:109E5000117F0B431377EAE708251828DCD1053D6D
:109E6000DAE7C046E865FF1FF0B58BB0059143887F
:109E70007E4F9E00F45915000493002C15D1012942
:109E800002D000200BB0F0BD101D57781678FFF7F8
:109E900057F9EB68320002932B7A049901930090F2
:109EA0003B002000FCF70CFFEBE7E388049A9342A9
:109EB00001D00820E6E72378012B00D1D4E0059BF0
:109EC000581E092800D9CFE001F06EFE05CE0A2900
:109ED000CC506C859AB229000498FFF773FFD1E744
:109EE000200029001022453001F086FDB9594B7839
:109EF000042B02D1013B4B70C3E70B000A00253352
:109F000035320C310498FFF795F90498FFF702FAFF
:109F10000522431E9841BB59C0005A70B2E7200089
:109F200029001022553001F067FD049B4F4C9D0025
:109F3000295904980A0006AB55320C31FFF77AF91B
:109F400029591022453106A801F0F6FD012808D153
:109F50000498FFF7F7F90590002804D106222B5941
:109F60005A7005988EE708230593FAE763780C2B5F
:109F70007AD1E36E002B03D11C2001F0A5FBE06633
:109F8000BB59D86E00286FD01022290001F034FD93
:109F9000BB590498DC6EFFF705FC0D22A076BB5977
:109FA0005A706EE7E06E00285ED063780D2B5BD1AF
:109FB0002B8808220382A91C123001F01DFDBB5919
:109FC0009A68517D0222114226D0186A407B1042C5
:109FD00022D00C32E4E763780E2B45D1236F002B9F
:109FE00003D1162001F070FB2067BB59186F0028C1
:109FF00003D01022290001F0FFFC0F22BB59CFE74C
:10A0000063780F2B30D1206F0622691C103001F0CD
:10A01000F3FCBB599A68517D0422114203D0196A9E
:10A02000497B1142D5D100210498FFF78BFA28E72C
:10A03000636F002B0DD0BB59586F0028F3D010224E
:10A04000290001F0D9FC0122BB5952425B6F1A6111
:10A05000E9E7142001F038FBBB5960675B6F002B08
:10A06000E9D126E72978DFE707200BE7E865FF1F3E
:10A0700010B5064C207001F07FFD06212078FDF719
:10A0800091FF0348FEF778FC10BDC046FB65FF1F3B
:10A090001192001100200BB270B50D00834216DA48
:10A0A000264B187801F0B0FB041E0DD00378922BDC
:10A0B0000ED0A02B37D0224B1878FF283AD02100A1
:10A0C00001F072FC002835D180200002684070BD8C
:10A0D00043780E2B0BD03E2BEDD18378052B12D07D
:10A0E000082BE8D181798088FFF7D8FA08E0154B72
:10A0F00082889A42DFD183681878591CFEF7C0FE27
:10A10000002817D1D7E7104B1B785B0712D50F4BF0
:10A110001B68002B0ED09B68002B0BD0C289811DC1
:10A1200080889847ECE7FFF741FAA068002801D043
:10A1300001F002FB200001F0A7FAC5E7FB65FF1F55
:10A140001943FF1F182000007564FF1FE465FF1FFF
:10A1500010B50078FFF712FA10BD10B50078FFF7C0
:10A16000FDFA10BD0C234343084A10B59B185A68EA
:10A17000002A03D0012901D1904710BD9B68002B14
:10A18000FBD00029F9D19847F7E7C0461866FF1FB2
:10A1900001238340094A10B5946B1C439463506BB0
:10A1A00098435063D46B20009843012901D12000CB
:10A1B0001843D063116B0B43136310BD0080004044
:10A1C000F0B500240127154B85B0DA6B144E0392CD
:10A1D0001A6C0192DA64019BE3403B4217D0039D65
:10A1E000E5403D400295E5B202992800FFF7BAFF2D
:10A1F000316A736A002908D03900002B01D0029916
:10A2000079402800FFF7C4FF01E0002BF9D10134A9
:10A210000C36172CDFD105B0F0BDC04600800040E1
:10A22000FC65FF1F064B01215A68C2400A4204D058
:10A230001B68C3401800084070471B6DF9E7C04613
:10A24000008000400122064B8240002903D0D968DB
:10A250000A43DA607047D9689143D960FAE7C0468B
:10A260000038004030B5032444430F4BE25C1B1917
:10A270009C785D7801232D1B0135AB40013BA34049
:10A28000A140DB430C00122807D80849920052185D
:10A29000116819402143116030BD054A11680B4017
:10A2A00023431360F8E7C046F7BE001108F00040F2
:10A2B00014F00040C21F70B5D4B20623092C0BD88D
:10A2C0000125084C9540002908D00021FFF7CAFF5E
:10A2D00023682B4323600023180070BD2368AB4321
:10A2E000F8E7C04600380040214BF0B51B185B78FA
:10A2F000022B21D1032444431E4A1F4EA35C121992
:10A300009478012215008540B76B013CE4B23D43CF
:10A31000A240B563194C122815D89B0000290CD116
:10A3200017495B1899680A439A600123205C154A13
:10A33000834011680B431360F0BD11495B189968A5
:10A3400091439960F1E70E4B00290DD159690A43F9
:10A350005A61225C1328E8D00123203A93400A492D
:10A36000086803430B60E7E7596991435961F0E7D7
:10A37000FC65FF1FF7BE0011008000403CBF0011CC
:10A3800000F00040A0F00040A4F00040F8B5002428
:10A390001B4E1C4D1C4B1B5D012B1FD1194A926992
:10A3A000E2401A420BD00122B25693402200143AE6
:10A3B000D2B2022A09D815494A6913434B610134C4
:10A3C00002360C35172CE5D1F8BD0022B2560F49E4
:10A3D0009200521891680B439360F0E7022BEED184
:10A3E000E7B23800FFF71EFF01235840C1B2380022
:10A3F000FFF77AFF3800FFF715FF6877DFE7C04601
:10A40000C9BE0011FC65FF1FFD65FF1F00F0004085
:10A41000012202388240054B002903D059690A43C2
:10A420005A617047596991435961FAE70038004011
:10A43000F8B50E0001210F008740114A0400D368CF
:10A44000FD43BB43D360831E8B4201D8FFF7E0FF7F
:10A4500000212000FFF72EFF0A4A0B4B5168012E06
:10A4600005D139431B1951605E700020F8BD2940A9
:10A47000516002221C1962709A6915409D61F4E7CF
:10A480000038004000800040FC65FF1F012210B52D
:10A490008240074B002906D019680A431A6001213F
:10A4A000FFF7C6FF10BD196891431960F7E7C04672
:10A4B000008000400C2370B5002543430A4A290060
:10A4C0009B181D70094B04001B185D70FFF7B0FF4F
:10A4D0000123A340064928000A681A430A60054977
:10A4E0000A689A430A6070BD1866FF1FFC65FF1F6B
:10A4F000348000403080004070B504000E00FF281A
:10A5000013D003250540FFF7D5FF084AA3089B0099
:10A510009B183F22ED00AA40AE40196820009143ED
:10A52000314319600121FFF78DFE70BD18380040DE
:10A53000F8B50C244443134B0500E4186368002B62
:10A5400003D1A3681220002B1AD0022201270E4B40
:10A5500000215B195A7028002770FFF769FF6368B4
:10A560001E1E08D0A3683E00002B04D02800FFF771
:10A5700059FE4640F6B228003100FFF709FE0020E0
:10A58000F8BDC0461866FF1FFC65FF1FF7B5C42065
:10A59000FF222B4B80001958002491433F3A0A4375
:10A5A0001A508022274F5202274E1A60274B1D5DFA
:10A5B000002D21D0A31E012B03D80121E0B2FFF70B
:10A5C00027FF012D18D11F4B9B69E3402B4213D06D
:10A5D000E3B218000193FFF725FE01000198FFF791
:10A5E00055FFE3B2143B022B1DD801217156184AC6
:10A5F0008D405369AB4353613B7F002B0DD0E5B2D7
:10A600002800FFF795FF2800FFF70CFE7B7F010075
:10A61000834202D02800FFF7A5FD01340C37023633
:10A62000172CC3D1F7BD012100237156F3568D407D
:10A63000074A9B009B189A68AA439A60DCE7C046C9
:10A6400000E100E0FC65FF1FC9BE0011FD65FF1FB2
:10A6500000F0004070B50E0015000400FFF72AFF5F
:10A660000C236343094A20009B189D605E60FFF73E
:10A670005FFFF021064B074A8900051E5A5002D0A1
:10A680002000FFF717FF280070BDC0461866FF1FA7
:10A690000000FF1FC1A1001170B5134D07202C78D9
:10A6A000002C1FD1982221005200280001F09CFAB2
:10A6B0000123C420FF222B700C4B80001C635C63C1
:10A6C0000B4B1C605C600B4B195891433F3A0A439B
:10A6D0001A50802252021A600D20074A074900F0E2
:10A6E000A3FF200070BDC046FC65FF1F0080004036
:10A6F000A0F0004000E100E08DA500118DA3001145
:10A70000030010B50620072B09D8054A137001F085
:10A710007BFAD7210020034B034A89005A5010BD11
:10A720004843FF1F0000FF1F911BFF1F70B51D0056
:10A7300002240C2910D8094ACA40D2070CD5FBF7CD
:10A7400041FF041E08D1059A04992800FBF756FF23
:10A75000FCF7C4FDFFF724FB200070BD12100000C1
:10A7600030B50D7802232C009C43184201D02B43B6
:10A770001C0008252300AB43284201D02B002343B3
:10A7800020241D00A543204201D01C4325002A237C
:10A790000D70184204D011781E3B0B43137030BD6E
:10A7A0000028FCD10C2113788B43F7E7F8B51D0086
:10A7B00006AB1B88140007AA0E000B201778002B8D
:10A7C00027D10A78022A49D14A68507811780002C4
:10A7D000244A08438018042840D801F0E5F9031200
:10A7E0001D1B2300F06800F05FFF021CC0B2B842DE
:10A7F00000D93A1CD2B22000F1682A8001F0FCF89E
:10A8000006E00222F3681B882A8023701B0A63700B
:10A810000020F8BD0622EEE701232B80F3681B78A9
:10A820002370F5E7F368002B16D008222A801A88D7
:10A8300022701A88120A62705A88A2705A88120A04
:10A84000E2709A8822719A88120A6271DA88A2717B
:10A85000DB881B0AE371DBE72B80D9E701202B8023
:10A86000D7E7C04600D6FFFFF7B516000A781D00EF
:10A8700008AB1F880C000123022A18D14A685078BF
:10A88000117800022B4A0843801803280FD801F0E2
:10A890008BF902254439E06800F006FFC0B20723B7
:10A8A000B84204D37B190193152B02DD0D23180048
:10A8B000FEBDE0682A003100C01901F09DF86B462A
:10A8C00000209B88E268D0541B4B1B68834203D056
:10A8D0001B68834200D098470023E8E70B23002F32
:10A8E000E5D1022DE2D1737832781B021343E2687E
:10A8F0001380114B1B68002BEED01B68002BEBD094
:10A900000120E8E70B23002FD1D1062DCED12A005C
:10A910003100E06801F070F8DEE70B23002FC6D1AC
:10A92000012DC3D132787533012AC0D8E3681A707B
:10A93000D2E7C04600D6FFFF0868FF1F70B50C00C5
:10A940001500072837D801F02FF9041436361B36C6
:10A95000242E182015290BD8184E1622002130005D
:10A9600001F03AF822002900300001F045F80020FB
:10A9700070BD18200229FBD11288114B1A80F6E70E
:10A9800018200829F4D10A000E48290000F01CFF05
:10A99000EDE718200129EBD10B4B10780B49DA6950
:10A9A000FFF7DEFEE3E718200129E1D1064B10781E
:10A9B0000749DA6BF4E70220DAE7C046F067FF1FC9
:10A9C000C643FF1FBC43FF1F4C43FF1F7443FF1FC1
:10A9D0009443FF1F030010B50020DB0704D50721B7
:10A9E000024A034800F08CF810BDC04654BF001165
:10A9F0004C43FF1F054A03001068002803D08288DB
:10AA00009A4201D1806870470068F6E7006AFF1F2C
:10AA10000A88030008009A4204D08A8804309A42C7
:10AA200000D0002070470000F8B5F22200230D4F3F
:10AA30000D4E7968050042433370994200D07B6027
:10AA40000A4C0021200000F0C7FF00231A007C60A0
:10AA5000AB4202D100203370F8BD01332280DBB25B
:10AA6000F234F5E7F86AFF1FF66AFF1F046AFF1F5A
:10AA700073B56B4601900600684615001980FCF717
:10AA80005FFF041E11D1002D0FD07689002E11D04A
:10AA90000C2000F019FE00280ED0084A046013684C
:10AAA00086808560002B02D11060200076BD1A00E0
:10AAB0001B68F7E70224F8E71324F6E7006AFF1F94
:10AAC000012100220A4B10B549420A4C1980998095
:10AAD0009A719A70084B2070012019805A60FFF714
:10AAE000A3FF2078FCF78AFF0448FDF745FF10BD5F
:10AAF0001068FF1F006BFF1FF86AFF1FADAB00114E
:10AB0000022310B5002802D0FFF7B2FF030018009F
:10AB100010BD0000030010B50020DB0704D50421A0
:10AB2000024A0348FFF7A4FF10BDC04668BF0011EA
:10AB3000CC43FF1FF0B50E2687B003930CAB1F88E4
:10AB400002ABF6180500080031000292FDF77AF812
:10AB500004000120002C0FD03088FFF74BFF0300CA
:10AB60000E20002B08D05E68002E05D021002800A2
:10AB7000039B029A0097B04707B0F0BD0A4B10B58F
:10AB8000984207D10122002352420A808B708A80AA
:10AB90008B7110BDFFF73CFF0028FAD001235B4208
:10ABA000038000238370F4E7FFFF0000F8B5050081
:10ABB00001290AD1134E00243388F227AB4219D061
:10ABC00028001149FFF7DAFF06E0022904D1013914
:10ABD000FDF750FF0028EDD0F8BD3B0063437268DD
:10ABE000D018D35A002B09D03A00002100F0F4FE0F
:10ABF0000134E4B2054B1B78A342EED801235B423B
:10AC00003380DDE7F86AFF1F1068FF1FF66AFF1F39
:10AC100010B5FFF7FDFE03000020834200D09878B6
:10AC200010BD0000F0B589B01C000EAB80CB0390C6
:10AC30001E8810AB1B78049202930B7A0D00DB0682
:10AC400016D42B780593022B24D00498FFF7D2FE5C
:10AC5000002812D003689C46002B0ED0029B2200D5
:10AC6000019329003B00644603980096A04705E045
:10AC70000498FFF7BFFE002802D10E2009B0F0BDF6
:10AC80008368002BF9D00A222900039898470028EE
:10AC9000D7D0F3E76B6858781A786B4B00021043F3
:10ACA0009842D2D8043B984210D2684B984242D086
:10ACB00015D8674BC0180128C7D80B20002EDDD14E
:10ACC000EB681A7859683A80200028E0614BC01878
:10ACD000032800D979E000F067FF846A789E5E4B14
:10ACE0009842B2D10B20002EC8D101233B80EB68E3
:10ACF00031001B7823706889013080B2FCF7A2FF15
:10AD00003A88031E0ED0017802328A183A804289AE
:10AD100062704289120AA27059680278E01C00F041
:10AD20006BFE06E004323A8031000422601C00F021
:10AD300053FE0020A2E70B20002E9FD1EB6807A94D
:10AD40001E8804233B80330A300026706370FCF7B2
:10AD500079FF051E28D004AB9A890E2304A95B183D
:10AD60003E49C668FCF7E2FF00280BD12B783C482F
:10AD70006A680599FBF798FB002803D1012304AA10
:10AD80005B42D3813278022A06D17168201D00F01F
:10AD900033FE3B8802333B800E2304AA9B181B889A
:10ADA000A3701B0AE370C4E704ABDE81F4E70B2059
:10ADB000002E00D062E7E9680398FFF729FF02231D
:10ADC0003B802070000A6070B3E70B20002E00D09B
:10ADD00054E70222EB681B883A8023701B0A6370D9
:10ADE000A7E7E86800F060FCC2B203000720B242A7
:10ADF00000D243E70DD00299DBB27118994202DB11
:10AE0000921BD3B20293029BE9681A003B80891916
:10AE10005AE70023F6E70B20002E00D02EE707228A
:10AE2000EB683A801A7822705A7862705A88A27059
:10AE30005A88120AE2701A792271DA886271DB8804
:10AE40001B0AA37175E7C046042900000228000010
:10AE500000D8FFFFFFD6FFFF03280000FFFF000020
:10AE600098BE0011F0B58DB06B46002008912022ED
:10AE70009B5E83423DDAA64B187800F0C5FC071EA6
:10AE800032D00378B02B2CD10079023816281FD885
:10AE900000F0E2FD17001E001E001E0031001E0023
:10AEA00096001E001D011E0052011E0073011E00AF
:10AEB000CD011E0050021E001E001E008E021E004C
:10AEC000E302944B94491B8878880B80FBF72CF89D
:10AED0003800FCF7ADFF914B1B68002B01D0380008
:10AEE0009847380000F0D0FB8020089B00024340C8
:10AEF00018000DB0F0BDEE220021874800F06CFD77
:10AF00000BAA3B7B7989388900923A000D32FCF715
:10AF1000B1FD0400804B1B78002C3FD146E0804BF4
:10AF2000788805937F4B4100CB5A0BAE073BDBB2D1
:10AF300032880293002301937B4B210006930093F8
:10AF4000059BFFF76FFE744D002810D1069B3A8ACF
:10AF50001B889A420BD138000599123000F0ECFDA5
:10AF6000002804D02B7862899B00EB185A801623A6
:10AF700006A81B18328820007989FCF7D7FE2B78A9
:10AF800004009A00AA1851880029C3D00133DBB20B
:10AF90002B70002807D006A9C98A9180634A1288BD
:10AFA0009A42BCD802E0012149429180002B04D092
:10AFB00059497888FAF7ECFF8AE73E890A2479E054
:10AFC00000253E89574B06937B88069A5B009B5A67
:10AFD000033B9D4202DB002DF0D05BE0162206A869
:10AFE00012183B7B798900923A0030000D32FCF751
:10AFF00041FD0590002858D04689017A7888FCF7F1
:10B0000003FD041E44D1464B78880793069B4100FC
:10B01000C95A454B0439C9B206AAD28A069302918D
:10B02000019400930599079BFFF7FCFD041E2FD1A7
:10B03000069B39491A88931C002D26D14B807988AC
:10B04000384B4900CB5A5119033B8B4220DD059BFD
:10B0500031485B8941190B71A91C0135C9B2EDB2A8
:10B06000059145191B0A2B71059B2D4904331818AE
:10B0700000F0C2FC2C4B059A1B88D318DDB22C4B78
:10B080009E4205D00136B6B29CE749889942D6D097
:10B09000002D0CD0204C2800618800F06DFC207041
:10B0A00021007888FAF784FF12E7059CF0E7002C6E
:10B0B00000D183E77B78142B00D109E716493B794F
:10B0C0004E800B700C717888FAF724FF00E7162485
:10B0D00006ABE41821003889FCF7B4FD011E00D14D
:10B0E000B7E1788822880F4C45002C5B0A4D013C63
:10B0F000E4B2029400240F4B01940095FFF792FDF7
:10B10000041E00D014E129007888FAF761FFDFE619
:10B11000006BFF1FB842FF1F1868FF1F0C68FF1F5E
:10B120000C69FF1F4864FF1FFC69FF1FB642FF1F29
:10B13000FFFF00001A68FF1F162406ABE418210069
:10B140003889FCF77FFD011E00D182E178882288D2
:10B15000AE4C45002C5BAE4D013CE4B202947C89C0
:10B16000AC4B01940095FFF75DFD041E00D0DFE0BD
:10B1700029007888FAF736FFAAE60025A44B1D803F
:10B180003B00F6331B78A24A78880792AB4208D975
:10B190009E4B12880693069943005B5A013B9A42E4
:10B1A00003DB0799FAF728FF92E616246B00FB18D9
:10B1B000059306ABE418059B21001889FCF742FDB6
:10B1C000011E03D1059B01241E8973E77888924BE9
:10B1D0002288069C099343001B5B904E013BDBB227
:10B1E0000293002300960193099BFFF71BFD041EA9
:10B1F00002D0059B1E895DE77B88069A5B009B5AFF
:10B20000079A108832881218934202DC1B1A013BFD
:10B2100033807F4C023032880999001900F0ECFB32
:10B220002388328801359B182380EDB2A8E70BAA4A
:10B230003B7B7989388900923A000D32FCF71AFC81
:10B2400000250590059B002B04D10A24002D00D178
:10B250006EE060E0059B7888197AFCF7D5FB010069
:10B26000041E63D1694C6C4B788806940993069B45
:10B270004400E45A694B063CE4B20BAE32880793B3
:10B280000294019100930599099BFFF7CBFC041EE2
:10B290004CD1079B5E491B881A1D002D30D14A8076
:10B2A000059B5B4C5A8963191A716B1C9BB2E3189E
:10B2B000120A1A71162306A832881B187989059874
:10B2C000FCF734FDFF21AA1C2E1D03350B00059051
:10B2D00092B2B6B2ADB2002803D006ABDB8AD9B2C7
:10B2E0001B0AA218651911712B714C4D301D2A884B
:10B2F0004949201800F080FB2B88F618B5B2A1E769
:10B300004988914207D17A8806995200525AEB181F
:10B31000053A9A42C4DC3E4C2800618800F03CFAB1
:10B32000207021007888FAF771FED1E5002DF2D166
:10B330003E89BFE6162606ABF61831003889FCF7C1
:10B3400081FC3D000400FA3500282DD0037A9B06CD
:10B350000CD400227B893989788800923A000C321B
:10B36000FFF7E8FB041E10D03E8915E03088FFF798
:10B3700041FB00281AD08368002B17D0210012222D
:10B3800078889847041EE4D0EEE72B78002B02D192
:10B390007888FAF74BFE00262B78002B00D097E533
:10B3A000002C00D194E585E60124DDE70E24DBE7DF
:10B3B000162506ABED1829003889FCF743FC041E5E
:10B3C00047D0037A9B0611D4154A7B88118899428D
:10B3D00003D01448814207D11380134BF2261D7805
:10B3E0000023D9B2A94221D30924A1E72888FFF775
:10B3F00001FB00282FD08368002B2CD021001222C3
:10B4000078889847041EDFD092E7C0464864FF1F43
:10B410001868FF1F1A68FF1F0C69FF1FFC69FF1FD8
:10B42000F86AFF1FFFFF0000F66AFF1F3100594353
:10B43000546801336018615A0029D2D13C000834A5
:10B440002100F22200F0D8FA21007888FAF7F6FD00
:10B450003EE501246CE70E246AE71D4B1A887B88C1
:10B460009A4231D07888FAF7F3FD31E5F223059856
:10B4700051684343CD18C95A00291FD03B7A012B8C
:10B480000BD16C88AB887888AA1D0094FFF752FB1B
:10B49000041E02D000233B722E88F22200212800D5
:10B4A00000F09AFA00232B80059B0133DBB2059351
:10B4B000084B05991B78064A8B42D7D801235B427B
:10B4C0001380002CCED0F5E5002634000596EFE77A
:10B4D000F86AFF1FF66AFF1F70B504000E00150022
:10B4E000FFF796FA031E08D131000548FFF790FADE
:10B4F00003001120002B02D01C8000209D7070BD25
:10B50000FFFF0000F8B50B4F06003B780D0014005C
:10B51000FF2B0ED00A2000F02FF9011E09D0B12315
:10B520000380002346800371C5800481387800F0D1
:10B530003BFAF8BD0D44FF1FF7B50F0008A9060040
:10B54000088809A90B240988002821D10234022B7C
:10B550001ED1557813782D021D432B008B43019388
:10B560007334002B14D1FB68300019000093FFF7EF
:10B570004FFB019C85420BD02A0030000099FFF759
:10B58000ABFF041E04D12A0030007989FFF7BAFF0F
:10B590002000FEBDF0B50E7885B003900AA805889E
:10B5A0000120022E0DD14C682778647824023C4398
:10B5B000054FBC4205D10398DBB201960095FFF719
:10B5C000BBFF05B0F0BDC04602290000034B10B51B
:10B5D0001B68002B00D09847FEE7C046046BFF1F96
:10B5E00007B501A8FFF7F2FF044A05480021121A27
:10B5F00000F0FAFAF8F706F9FEE7C046086BFF1FFD
:10B600001044FF1F0000000001B40248844601BC42
:10B61000604700BFC9A9000001B40248844601BCCC
:10B62000604700BF5522000001B40248844601BCB7
:10B63000604700BF1131FF1F01B40248844601BCBE
:10B64000604700BF156B010001B40248844601BC8D
:10B65000604700BFFD38FF1F01B40248844601BCAB
:10B66000604700BFA54F010001B40248844601BCF9
:10B67000604700BF8D12000001B40248844601BC3F
:10B68000604700BF091B000001B40248844601BCAA
:10B69000604700BF434D010001B40248844601BC2D
:10B6A000604700BFE548000001B40248844601BC81
:10B6B000604700BFDD52010001B40248844601BC6E
:10B6C000604700BF014C010001B40248844601BC40
:10B6D000604700BF3D4B010001B40248844601BCF5
:10B6E000604700BF2124000001B40248844601BC29
:10B6F000604700BFED4A010001B40248844601BC26
:10B70000604700BF8552010001B40248844601BC75
:10B71000604700BF9D3AFF1F01B40248844601BC48
:10B72000604700BF8B52010001B40248844601BC4F
:10B73000604700BF311B000001B40248844601BCD1
:10B74000604700BFD949010001B40248844601BCEA
:10B75000604700BF456B010001B40248844601BC4C
:10B76000604700BF056A000001B40248844601BC7E
:10B77000604700BF3539FF1F01B40248844601BC51
:10B78000604700BF1D4D010001B40248844601BC62
:10B79000604700BF2951010001B40248844601BC42
:10B7A000604700BF090E000001B40248844601BC96
:10B7B000604700BFC94A010001B40248844601BC89
:10B7C000604700BF055E000001B40248844601BC2A
:10B7D000604700BF810E000001B40248844601BCEE
:10B7E000604700BF5549010001B40248844601BCCE
:10B7F000604700BF7539FF1F01B40248844601BC91
:10B80000604700BF5125000001B40248844601BCD6
:10B81000604700BFF54E010001B40248844601BCF8
:10B82000604700BFF30E000001B40248844601BC2B
:10B83000604700BF0934FF1F01B40248844601BCC1
:10B84000604700BF291C000001B40248844601BCC7
:10B85000604700BF090E000001B40248844601BCE5
:10B86000604700BF75A9000001B40248844601BCCE
:10B87000604700BFB352010001B40248844601BCD6
:10B88000604700BFE938FF1F01B40248844601BC8D
:10B89000604700BF1147010001B40248844601BC63
:10B8A000604700BFF94C010001B40248844601BC66
:10B8B000604700BF6DBC000001B40248844601BC73
:10B8C000604700BF4550000001B40248844601BCF7
:10B8D000604700BF3D18000001B40248844601BC27
:10B8E000604700BF4137FF1F01B40248844601BCD6
:10B8F000604700BFADAE000001B40248844601BC01
:10B90000604700BFF537FF1F01B40248844601BC01
:10B91000604700BF3519FF1F01B40248844601BCCF
:10B92000604700BF4D1F000001B40248844601BCBF
:10B93000604700BFE117000001B40248844601BC23
:10B94000604700BF8930FF1F01B40248844601BC34
:10B95000604700BF7136FF1F01B40248844601BC36
:10B96000604700BF9DA9000001B40248844601BCA5
:10B97000604700BF0919FF1F01B40248844601BC9B
:10B98000604700BF350E000001B40248844601BC88
:10B99000604700BF350E000001B40248844601BC78
:10B9A000604700BFB54C010001B40248844601BCA9
:10B9B000604700BF594F010001B40248844601BCF2
:10B9C000604700BF5D17000001B40248844601BC17
:10B9D000604700BF2146010001B40248844601BC13
:10B9E000604700BF154D010001B40248844601BC08
:10B9F000604700BF213AFF1F01B40248844601BCE2
:10BA0000604700BFE94C010001B40248844601BC14
:10BA1000604700BF7130FF1F01B40248844601BC7B
:10BA2000604700BF691F000001B40248844601BCA2
:10BA3000604700BFA946010001B40248844601BC2A
:10BA4000604700BF312EFF1F01B40248844601BC8D
:10BA5000604700BFC51D000001B40248844601BC18
:10BA6000604700BF353BFF1F01B40248844601BC5C
:10BA7000604700BF5147010001B40248844601BC41
:10BA8000604700BF0D52010001B40248844601BC6A
:10BA9000604700BFF13AFF1F01B40248844601BC71
:10BAA000604700BF4136FF1F01B40248844601BC15
:10BAB000604700BF6571010001B40248844601BCC3
:10BAC000604700BF4551010001B40248844601BCF3
:10BAD000604700BFB132FF1F01B40248844601BC79
:10BAE000604700BF0D3BFF1F01B40248844601BC04
:10BAF000604700BFE928000001B40248844601BC49
:10BB0000604700BF2526000001B40248844601BCFE
:10BB1000604700BF4D36FF1F01B40248844601BC98
:10BB2000604700BF5952010001B40248844601BC7D
:10BB3000604700BFC56D010001B40248844601BCE6
:10BB4000604700BFCD4C010001B40248844601BCEF
:10BB5000604700BFEDA5000001B40248844601BC67
:10BB6000604700BFB539FF1F01B40248844601BCDD
:10BB7000604700BFD91B000001B40248844601BCE5
:10BB8000604700BFC926000001B40248844601BCDA
:10BB9000604700BF7918000001B40248844601BC28
:10BBA000604700BFB14E000001B40248844601BCAA
:10BBB000604700BF213BFF1F01B40248844601BC1F
:10BBC000604700BF851F000001B40248844601BCE5
:10BBD000604700BFC521000001B40248844601BC93
:10BBE000604700BF0124000001B40248844601BC44
:10BBF000604700BFB70E000001B40248844601BC94
:10BC0000604700BFD932FF1F01B40248844601BC1F
:10BC1000604700BF911BFF1F01B40248844601BC6E
:10BC2000604700BF017F000001B40248844601BCA8
:10BC3000604700BFC93AFF1F01B40248844601BCF7
:10BC4000604700BFDD66010001B40248844601BCC4
:10BC5000604700BF3555000001B40248844601BC6E
:08BC6000604700BF1D4B01000D
:10BC680000030102020303030403050006020700A0
:10BC7800080209030A030B030C000D000E030F034F
:10BC8800100311031303140315021602B13B00112C
:10BC9800E53B00110000000002000000AABC0011F2
:10BCA800192A0F180A000000F1590000FD240000AD
:10BCB800414601008180001195A00011E97400112E
:10BCC800857E00112D53001165AE0011794F0011CA
:10BCD800C13D0011F13E00110000000016160000E1
:10BCE80002000000F4BC0011F4FFF3FFD2FC0000D6
:10BCF8003140001100000000000000005475796117
:10BD08000042312E3900303031410067697468755E
:10BD1800622E636F6D2F7076767800544842330038
:10BD2800020000003CBD0011292A282A272A262AB9
:10BD3800252A242A0A180000E204000071020000E3
:10BD480078EC000005000000744000001027000097
:10BD580060F000000400000006640000204E0000AF
:10BD68000000000006000000050000001F501D0034
:10BD7800023CB40000011A0019000000A1020000F2
:10BD88003031323334353637383941424344454609
:10BD98000000000031570011855700110000000015
:10BDA80002000000B4BD00116F2A6E2A1A18EAD8E2
:10BDB800BC80F0FC600000000000000000005F068E
:10BDC8006B2F363D7D077F3F777C596E7971000078
:10BDD80001A00000000000006410B71DC8206E3BE1
:10BDE800AC30D9269041DC76F4516B6B5861B24D7A
:10BDF8003C7105502083B8ED44930FF0E8A3D6D6E4
:10BE08008CB361CBB0C2649BD4D2D38678E20AA04B
:10BE18001CF2BDBDFB349B5F800000800010000059
:10BE280000000000EB600011757700110F61001130
:10BE38007D7B001193610011537B00110962001191
:10BE4800297B00115B620011F17C0011C3620011B3
:10BE5800F17C0011F5620011AB7C00110962001140
:10BE6800E17A001181620011897C00110000000054
:10BE78000000000067630011897C0011C96300118C
:10BE88008D770011052A042A012A002A022903288D
:10BE98000128002801180018000000000000000018
:10BEA80000000000000000870101020102010102F8
:10BEB800010203030401030101010101030302015B
:10BEC80003000D000E0010001100130014010701FB
:10BED80008010A010B011C011D02040205020702E8
:10BEE800080219021A021C021D03010302031700AB
:10BEF8000201000504000807000B0A001716001DC0
:10BF08001C010201010504010E0D01111001141399
:10BF1800011716011A19020201020B0A020E0D027C
:10BF28001110021413021716030504030807030B64
:10BF38000A030E0D0001020307090A0B0E0F101168
:10BF480012141718191A1B1F20212200ADA700115F
:10BF580069A8001100000000020000009EBE001148
:10BF68000000000095B5001100000000020000006C
:04BF78009CBE00115A
:020000041FFFDC
:1000000000000000293D0011B0BC0011ACBC001183
:100010004061FF1F00000000000000000000000021
:1000200000000000000000000000000000000000D0
:1000300000000000000000000000000000000000C0
:1000400000000000000000000000000000000000B0
:1000500000000000000000000000000000000000A0
:100060000000000000000000000000000000000090
:100070000000000000000000000000000000000080
:100080000000000000000000000000000000000070
:100090000000000000000000000000000000000060
:1000A0000000000000000000000000000000000050
:1000B0000000000000000000000000000000000040
:1000C0000000000000000000000000000000000030
:1000D0000000000000000000000000000000000020
:1000E0000000000000000000000000000000000010
:1000F0000000000000000000000000000000000000
:1001000000000000000000000000000000000000EF
:1001100000000000000000000000000000000000DF
:1001200000000000000000000000000000000000CF
:1001300000000000000000000000000000000000BF
:1001400000000000000000000000000000000000AF
:10015000000000000000000000000000000000009F
:10016000000000000000000000000000000000008F
:10017000000000000000000000000000000000007F
:10018000000000000000000000000000000000006F
:10019000FD32FF1F5D31FF1FC1660100000000003E
:1001A000000000000000000000000000000000004F
:1001B000000000000000000000000000000000003F
:1001C000000000000000000000000000000000002F
:1001D000000000000000000000000000000000001F
:1001E000000000000000000000000000000000000F
:1001F00000000000000000000000000000000000FF
:1002000000000000000000000000000000000000EE
:1002100000000000000000000000000000000000DE
:1002200000000000000000000000000000000000CE
:1002300000000000000000000000000000000000BE
:1002400000000000000000000000000000000000AE
:10025000000000000000000000000000000000009E
:10026000000000000000000000000000000000008E
:10027000000000000000000000000000000000007E
:10028000000000000000000000000000000000006E
:10029000000000000000000000000000000000005E
:1002A000000000000000000000000000000000004E
:1002B000000000000000000000000000000000003E
:1002C000000000000000000000000000000000002E
:1002D000000000000000000000000000000000001E
:1002E000000000000000000000000000000000000E
:1002F00000000000000000000000000000000000FE
:1003000000000000000000000000000000000000ED
:1003100000000000000000000000000000000000DD
:1003200000000000000000000000000000000000CD
:1003300000000000000000000000000000000000BD
:1003400000000000000000000000000000000000AD
:10035000000000000000000000000000000000009D
:10036000000000000000000000000000000000008D
:10037000E1B50011000000000000000000000000D6
:10038000000000000000000000000000000000006D
:10039000000000000000000000000000000000005D
:1003A000000000000000000000000000111BFF1F03
:1003B000000000000000000000000000000000003D
:1003C000000000000000000000000000000000002D
:1003D000000000000000000000000000000000001D
:1003E000000000000000000000000000000000000D
:1003F00000000000000000000000000000000000FD
:08183800106FFF1F4118FF1F94
:10184000024981F3088802F0F7FA0000106FFF1FC9
:1018500070B500241E491F4A1F484C6308CA1B0567
:101860001B0DE4188242F9D11C4B80228B630021AE
:1018700009201B4B920519621A4B1B4DDA671B4B53
:10188000DA688243DA609A68194802409A60112047
:10189000296002F08FF8112002F06CF86B6C154A89
:1018A000112013406B64EE23DB006343124A1B0CD0
:1018B00013840122114B9A7201F006FC104B1B7825
:1018C000002B04D10F4B1021187802F025FA70BDBF
:1018D000000005400806054080060540FF010000A5
:1018E00000F0004004E100E0003800403CF000401F
:1018F000FFDFFFFFFFFEFFFF1061FF1FC461FF1F3F
:10190000F263FF1FF061FF1F10B502F025F90728F1
:1019100004D0122808D0022808D010BD044A0420A0
:10192000136B01331363F8E70220F6E71420F4E7A2
:10193000F064FF1FF8B507000C00260025005036A4
:1019400030785135002804D10300287058342370B2
:10195000F8BD2978CA00481E8141A3183800A25C4E
:101960005B68C9B2FFF7D0FF00280DD12B78DA00F1
:10197000A218013350602B703378044A013B337056
:10198000136A01331362D8E70123DFE7F064FF1F16
:101990005C234343074910B5C9180B0058331B7823
:1019A000012B05D1FFF7C6FF034A936A0133936207
:1019B00010BDC0462465FF1FF064FF1F10B502F084
:1019C00033FB064A0121130010CB4942D967044B6F
:1019D000136002F049F9200010BDC04600E100E0AC
:1019E0001000100010B5040002F01EFB024B1C603A
:1019F00002F03AF910BDC04600E100E0431E5A4231
:101A00005341A022F0B5D2015B421340154D164A56
:101A100040019B182A18127E8BB00191002A1BD01E
:101A20001A000832D46F0022E6B206AFE4B2944244
:101A30000EDC2818C369002B08D0019902AA117185
:101A400006AA049202AA167303A898470BB0F0BD29
:101A50001978B9540132EAE71A7D1A7806AB0126E3
:101A60001A70E6E7B067FF1F00400040F0B5254B55
:101A700004004001C25C85B0002A2BD01A18117EE8
:101A8000002927D0917E002924D01179022921D163
:101A90001689D788D168F51BADB22A1C102D00D944
:101AA000102292B2BE4217D11818012303710023ED
:101AB000C269C38003819A4206D06846032103733A
:101AC0000171029301A890470820002C00D0192032
:101AD00001F0FAFA05B0F0BD013C65426C41A02569
:101AE0006442ED012C40084D1B186419074D063364
:101AF000013A92B2AA42EDD01888461C1E80085CBA
:101B00002070F5E7B067FF1F00400040FFFF0000B6
:101B10000F220E4B10B59868104002380A280BD8D7
:101B200001F0FEFF0D0A0B0A0A110A0A0A0A060052
:101B300002210020FFF762FF10BD0121F9E700201C
:101B4000FFF794FFF8E7DB6FF6E7C0460040004080
:101B50000F220E4B10B59868104002380A280BD897
:101B600001F0DEFF0E0A0B0A0A120A0A0A0A060030
:101B700002210120FFF742FF10BD01210800F9E713
:101B80000120FFF773FFF7E7DB6FF5E700900040F8
:101B900013B5334C2378072B3DD8324B1A78324B90
:101BA000002A39D18022196852020A431A6025207E
:101BB00001F0C0FE20232D4A11680B4380211360E1
:101BC0006B460422C90508680733104228D08021DB
:101BD0000422C905C86810422ED080212020C905E2
:101BE000CA688243CA6014221A701A78002A2FD158
:101BF0008021C905C86820320243CA6014221A70C5
:101C00001A78002A28D11A4B1A7D22785A601D2290
:101C10001A705932DA6013BD1A6816490A40C5E7CE
:101C2000086802430A6014221A701A78002ACED07B
:101C30001A78013AD2B2F7E7C8680243CA601422A0
:101C40001A7019784A1ED2B21A700029F9D1C4E765
:101C50001A78013AD2B2C7E71A78013AD2B2CEE77F
:101C60004843FF1F1044FF1F3CF000404043FF1F4C
:101C700000200040FFFFFEFF564B70B51B68012B94
:101C800003D1554A936D0133936502F08DF9534B9F
:101C9000534A1860534B544C1A600123534A136043
:101CA000534A13602378002B06D00622514952482C
:101CB00001F072FF00232370504A514B10681B78CB
:101CC000C1B2002B0ED14F4CC0B223785BB2002BB7
:101CD0004FDB237824785BB264B21B0424021B1907
:101CE0001B1813600B1C50294ED95023464A4749F4
:101CF0001078DBB2FF2202284BD10868444C454DD6
:101D0000267890432A78964254D9227824782E78DF
:101D1000023B5D10A31B6B435201D31A10335B11BE
:101D20001843086001F070FF031F012B45D83A4BA0
:101D30001B78002B06D0394B1B78002B02D00020DB
:101D400002F01AF9A122364B92009978354B4A439A
:101D50001B689B18832292009B181B78033B012B66
:101D600003D8AF20400002F03FF901222E4BDA8267
:101D700070BD237824785BB264B2FF33FF341B0458
:101D800024021B190138ABE7CAB2022AAED20223E1
:101D9000ACE70868254C264D267890432A78964271
:101DA00008D9227824782D78023B5B10641B6343AA
:101DB0005201B2E72378DBB2B2E70228D5D11D4B3E
:101DC0001B78013B022B03D91B4B1B78022BCCD178
:101DD0006C20C8E79809FF1FFC0FFF1F3C64FF1F22
:101DE000FF3F0000141003404064FF1F0C1003402D
:101DF00000100340D50BFF1F7211FF1FB4000340FA
:101E00008C09FF1F680AFF1F490AFF1F9400034047
:101E1000460AFF1F470AFF1FF908FF1F2209FF1F7D
:101E2000300DFF1F3409FF1FBC0BFF1F440AFF1FAB
:101E3000450AFF1F1C09FF1F2309FF1F10B502F0F1
:101E400033F80022014B1A8010BDC0463A64FF1FD0
:101E500010B502F041F8A121054A89009478054A9D
:101E600061431268044B5218528C1A8010BDC04650
:101E7000300DFF1F3409FF1F3A64FF1F10B50D4BD3
:101E80000D4A9978A1239B004B431268D218531D29
:101E9000D97F0A4B1B88994209D2441C07D0C82815
:101EA00005D0D2695B1A5A43054B5343C01801F061
:101EB0000BFF10BD300DFF1F3409FF1F3A64FF1FD9
:101EC0007102000070B5244D2B68002B28D001F062
:101ED00033FF2B68D8402B680400002B27D001F07B
:101EE00053FE2B68D8401D4B1D4A9978A1239B00B7
:101EF0004B431268D118D25C91239B00002A20D05A
:101F0000CA580132CA50174B17491B6808688342E8
:101F100014D3D23B181A012A1AD0144B186070BD82
:101F200001F00AFF124B196801F026FED3E701F019
:101F30002BFE0F4B196801F01FFED4E70D495B180B
:101F4000E8E7CA500C4B1B68DB68E418201AE4E78A
:101F5000F530FF30E1E7C0461C08FF1F300DFF1FC2
:101F60003409FF1F9C09FF1F3C64FF1FA009FF1FCE
:101F70001808FF1F2DFF3F004464FF1F70B50400C9
:101F80000D00282916D10300A433C2881B889B1A90
:101F90000B4A9BB293420DD906006A3605223100E6
:101FA000653001F051FF002804D13100200001F01C
:101FB0004BFE70BD2900200001F0C6FEF9E7C046C7
:101FC000FE7F0000F8B50500012001F095FF134CDD
:101FD000A36AA26A9342FBD1114E336001F08CFEDA
:101FE0001049030008601048426894460F4A176879
:101FF0000022BC4501D24268BA1A0D48026032681C
:10200000AD18A422E562606A520302436262094A83
:102010001278002A01D00F3B0B60F8BD00F00040A1
:10202000340AFF1FE408FF1F28100040180AFF1F92
:102030001C0AFF1F1C09FF1F70B580241025E40532
:10204000A3682B43A36001F0C7FEA368AB43A36062
:1020500070BD0000F7B5160080221C001023D205C9
:102060000191916805000B43936000225A4BD730D1
:102070001A6001F079FD9D232A002F009B00EB5888
:10208000CA3201210092FC37002B01D00021009AB6
:10209000386801F0E1FD2900009BCB311A784F4BE5
:1020A000D3351A604B780A781B0213438A781204DE
:1020B0001A43CB781B061343494A1BBA13604B796A
:1020C0000A791B0213438A7912041A43CB7931002F
:1020D0001B061343434A1BBA13606B782A781B0212
:1020E0001343AA7812041A43EB781B0613433E4AA3
:1020F0001BBA1360019A330213433C4A13603C4BF2
:1021000022001B1B9C4603293DDCB3089A001300E8
:102110005142B21A032A46D1354AE018511A827840
:102120004078120400020243E05C043302430A6078
:102130000022FF2B4BDDF0222E4B12011A600F22E2
:102140002D4B1A602D4A1368002BFCD00023224A25
:1021500027491360091B321D0B191B68043A180A22
:1021600023706070180C1B0EA070E3700434002AFA
:10217000F2DC802210213B68D20501333B6093687A
:102180008B439360F7BD6346D578981893782D06F6
:102190001B042B43157804392B43557804322D0248
:1021A0002B430360AFE7022A0AD1114AE05C511ABF
:1021B000E2185278120202430A6004339BB2B7E776
:1021C000012AB5D10A4A521AE15C1160F5E70849C3
:1021D00059180A600433ACE7000004403C00044096
:1021E0003800044034000440300004400C00044037
:1021F00000010440040004401000044014000440A6
:10220000F7B5150080221C001023D20500919168BB
:1022100007000B4393600023654AD730136001F039
:10222000A3FC9D233E009B00F9583B00CA363200B8
:10223000FC33002900D07FE0586801F00DFD390023
:1022400032785C4BCB311A604B780A781B0213430F
:102250008A78AC4612041A43CB78281D1B06134318
:10226000554A1BBA13604B790A791B0213438A79CA
:1022700012041A43CB791B061343504A1BBA13604E
:102280004B7A0A7A1B0213438A7A12041A43CB7AD6
:1022900021001B0613434A4A1BBA1360009A2B0203
:1022A0001343484A13602200474B1B1B0093009BBB
:1022B000CE785B1801938B7836061B0433430E7877
:1022C000043833434E78043136023343019E336081
:1022D0000328ECDC0321A808431C9B002940800054
:1022E00003292BD13849E5185E18A9786D78E35C8D
:1022F00009042D02294319433160030008330021EA
:10230000FF2B2DDD314B324919600F21314B196004
:10231000012327490B60304B19680029FCD00621A6
:102320001B680B40042B20D080220020D20593682C
:102330000A318B439360FEBD01217DE7022908D15C
:1023400021495D18E1184978E35C090219432960C5
:10235000D3E70129D3D11C495918E35C0B60CCE7C2
:102360001948181801600433CAE7002310490B60AC
:102370006346002B0CDC3B00FC335A681021013211
:102380005A608022D205936801208B439360D2E784
:10239000009B9B181B68190A13705170190C1B0EB7
:1023A000D37004235B4291709C440432E0E7C04642
:1023B000000004403C000440380004403400044065
:1023C000300004400C0004400001044004000440BC
:1023D000080F0000100004401400044070B5061EF1
:1023E00019D002225A4B9B799343012B13D1594B9D
:1023F0001A78FF2A0FD15A78FF2A0CD19A78FF2A2F
:1024000009D1DA78FF2A06D11A79FF2A03D15B793C
:10241000FF2B00D199E0504B0C201A78012A08D0EC
:1024200000224E4D1A7029780B00093B042B01D86D
:10243000212070BD4B1F012BFAD9454CA37B042BE7
:1024400000D982E0A279032A00D97EE09A1ED2B296
:10245000012A02D860881F2877D9002E56D0012E75
:1024600073D1A0880128E3D0002907D1581E032882
:1024700003D801F055FB121715122E702978481E4B
:10248000032811D80025364B1D602823237501F041
:10249000B3FBA84227D0A580CAE702212970EDE747
:1024A0000421FBE70321F9E707390129C0D82D49A9
:1024B0000968C96A8906BBD52B4908780028B7D1B5
:1024C000012A01D9002BB3D102230B708021274DA3
:1024D000263389012878237501F016FC802128789D
:1024E000890101F019FC0123A380214B1B78002BEB
:1024F0000AD0FA2280211F4B92001B8809025A43FE
:102500001A4B187801F088FD002092E701F08CFD4D
:102510002B78A680073B012B03D917482E7001F0BA
:10252000C3FB114B114C1A78002A06D080210022DF
:10253000207889011A7001F0E7FB01F095FB8021FA
:102540002078090201F0E0FBDEE7122071E7C046C7
:10255000A60BFF1F6B09FF1F1A09FF1F1C09FF1F96
:102560004809FF1F4464FF1F2309FF1F1B09FF1FAA
:102570002109FF1F2C09FF1F0010004010B5002982
:1025800001D001F079FB10BDF7B5604B019199784E
:10259000A1239B004B435E4A060014681022E418F6
:1025A000D6235B00E0583623FF33E35C00279343D8
:1025B000222B41D1574B0F3A1A600760012501F0D9
:1025C00003FC019B1880E8235B00E35C002B01D037
:1025D000B34258DD0023504FFB70AD33FF33E35857
:1025E0001A68002A03D09B88DB439B071DD0382341
:1025F000FF33E35C002B18D09B235B00E35C002BD4
:1026000013D1D133FF33E35CB3420EDAA4235B0072
:10261000E15AE018090A023101F08EFC2300012280
:10262000FE33013E01351A87FA70E8235B00E35C54
:10263000002B2AD0A8B2FEBD03683D00002BBED0FF
:1026400081880430090A023101F076FCD6235B0050
:10265000E3581F60B2E72300B133BA00FF33985844
:10266000013781880430090A023101F065FCE82352
:102670005B00E35CBB42EEDCE822F61AED180023B7
:102680005200A354A6E70027F1E7200001F04CFB1D
:1026900000281FD0002E1DDD7319882647190193CD
:1026A000B600200001F018FB5A3080002018406866
:1026B000013581880430090A023101F03DFC200017
:1026C00001F04AFBA3590133A351BD4202D0019B43
:1026D0009D42E6D1114BE35C002BABD095239B00D0
:1026E000E35C002BA6D00E4BE15A0029A2D00D4A84
:1026F000A35C994202D90133A3549BE700231A211A
:102700002000A35401F058FB94E7C046300DFF1F92
:102710003409FF1F00140340E010FF1F5A0200009D
:10272000720200005E0200000D4970B54A6E0D4C49
:10273000D2038B69D20BA24206D80B4D0224AA42C7
:1027400004D901F041FC70BD02246442E218150076
:102750007E2425402242F4D0A3432B438B61F0E733
:1027600000F000400A200000FC1C0000F8B51D4BE2
:102770001D4F1A78002A10D1BA7B002A02D10132EB
:102780001A7003E0032AFAD0022AF8D001F034FAD2
:1027900000220120154B1A70F8BD154B154D1C6811
:1027A000154B9E7801232B702878C0B200F09EFB59
:1027B000BB7B002B0BD101F017FAA1239B007343C5
:1027C000E41883239B00E41823782B70E4E7032BA1
:1027D00002D101F019FBF0E70020022BDCD101F05F
:1027E000B3F9EAE71C09FF1FA60BFF1F2309FF1F10
:1027F0003409FF1F490AFF1F300DFF1FF0B587B0D6
:102800000EAD2F780FAD2D780593AC4663461400BE
:102810000E4D0CAA12782E7803930D9B0092019313
:102820002200059B029701F0E7FA2E70012C01D0DF
:10283000042C08D1802206498B889343054A1278DC
:10284000D20113438B8007B0F0BDC0461C09FF1FA7
:102850006C11FF1F7809FF1F0B001B3B70B50400B4
:102860003020E02B0DD81300E025493BFF3B9BB205
:10287000ED00AB4205D8034B200019825A8201F0CB
:1028800083FA70BD8410FF1F10B501F08DFB054B5E
:1028900000205B68052B04D9034A5268D20200D499
:1028A000980810BD00100040FCE100E070B501F098
:1028B000BBFB0D4B1B68FC33DC691D6AFFF7E4FFB3
:1028C0006419844204D2094B01241B68002B07D0F1
:1028D00004220024064B1A70064A9369013393615F
:1028E00001F0C2F9200070BD4464FF1F9809FF1F6A
:1028F0002309FF1FFC0FFF1F70B50C4D2B68FC3325
:102900005C6A01F091FBFFF7BFFF2B680025FC33E9
:102910009B6AE318834204D2054B1B68AB4200D18B
:10292000051B01F0A1F9280070BDC0464464FF1FDB
:102930009809FF1FD722044B92009B5810B5002B1B
:1029400000D0984710BDC0460000FF1F10B501F031
:10295000CFF8FFF7EFFF2749274BCA6D274C1A40E6
:1029600084235B001343CB65254B1B68186A01F079
:10297000C3FA244B244A1A60244B254A1A60A02229
:10298000244B52001A60244B187801F0BDFA200045
:10299000224901F001FA0023A3600233A360204B17
:1029A0002049236003232048A36001F0F5F9102299
:1029B0001E4BFF201A60802252031A60802292036D
:1029C0001A60802212041A6001F0D6FA012001F088
:1029D0008BF9FA20400001F047FA582001F004FB7F
:1029E000134801F019F9012001F0E6F8072001F081
:1029F0009BFA10BD00F0004000FEFEFF14100040E6
:102A00004464FF1F000003400180063DBC000340FA
:102A100034080000A40003404A0AFF1F71020000AE
:102A2000C3090000FFFF3F002810004000E100E064
:102A300030750000674E336888331B6883F308885D
:102A400001F01AFA644A6549136800200B401360CC
:102A5000634B644A1B68934200D1A6E001F0BCF8C6
:102A60000221614A13688B431360FFF76FFF5F4BCE
:102A70005F4C1878C0B201F0BFFA0023A3600233A4
:102A8000A3605C4B0120236001F036FA0323A360AE
:102A900001F012FA040001F087FA050001F00CFAC7
:102AA000554B186001F0B8F9544B1968621A531E5F
:102AB000A14200D213008022D203934201D39B0291
:102AC0009B0A3268D16AC90700D471E04C491C0CDA
:102AD00009689BB24C4359432402090A641803262F
:102AE0004849FC3293680A6847489B1A474A076876
:102AF000126847499B18474A9A1833409208DB19D5
:102B00000A600360042B03D9013233400A6003607A
:102B10000E684149A619300001F02EF83F4F3E499A
:102B20003B68C3183B603000019301F095F93C4EBF
:102B30003068081838493060884205D9019B013354
:102B40003B6001F089F9316001F076FA354B1B7872
:102B5000002B0DD001F028FA334B621B19681218B4
:102B60008A4232D24919091B091A304801F014F976
:102B70002F4E337A002B0ED001F016FA621BF1684B
:102B80001218914224D94919091B091A294801F040
:102B900003F900233372284B83F3088801F0ECF823
:102BA000002001F019F801F00FF801F015F85CE7CA
:102BB000DC0199000234641A5900641A09214B435C
:102BC0008033CB40A408E41889E7FA218900CCE7D8
:102BD0001A49DBE74464FF1F1CF00040FFFFC1FF00
:102BE0000C0AFF1FB641210310000040490AFF1FD5
:102BF00014100040C3090000100AFF1F340AFF1F11
:102C0000380AFF1F200AFF1F280AFF1F1C0AFF1F88
:102C1000240AFF1FC4090000710200006008FF1FA2
:102C20002C0AFF1F1C09FF1FE408FF1F00100040B3
:102C3000740BFF1F3C10004000000020DC0500006A
:102C4000A022054B92009B5810B5002B01D098474D
:102C500010BD01F0C1F9FBE70000FF1FA122054BE9
:102C600092009B5810B5002B01D0984710BD01F081
:102C7000B3F9FBE70000FF1FA222054B92009B580F
:102C800010B5002B01D0984710BD01F0A5F9FBE766
:102C90000000FF1FA322054B92009B5810B5002B8C
:102CA00001D0984710BD01F097F9FBE70000FF1F26
:102CB000A422054B92009B5810B5002B01D09847D9
:102CC00010BD01F089F9FBE70000FF1F70B501F0AE
:102CD0006BF94F4B186001F067F80400C30702D48A
:102CE00001F0DAF870BD00224A4B1A604A4B18789E
:102CF0000138042829D800F013FF0320181C2400F1
:102D0000200000F051FF0128ECD0444C2378042B24
:102D10006ED101F0E9F80028E4D001F03DF9582027
:102D200001F062F902232370DCE7200001F044F98E
:102D3000E9E7200001F018F8E5E7200001F024F9A8
:102D4000E1E7200001F0C0F8DDE700F05DFF0500DD
:102D5000012808D1324B1B78053B012B03D82000FA
:102D6000FFF76EFFD1E72D4B1B78022B01D0052B0F
:102D700020D1022D28D12B4B9B7BAB431CD12000B3
:102D8000FFF76CFF264B18780128BED16405BCD430
:102D9000244925224B7B034205D1233A13405A4252
:102DA000534126331A000B7D9342AED9322001F0F5
:102DB000D3F8AAE7022D07D1194B1B78052B11D1A7
:102DC0002000FFF759FFDDE7012D0BD1012B03D1C7
:102DD0002000FFF75FFF98E7062B03D12000FFF7E5
:102DE00067FF92E7200001F0F7F8022D8DD1C9E7C7
:102DF000032B04D10C4B987C00F0F6FF72E7072BF5
:102E000000D06FE7094B987B00F03EFF6AE7C046B1
:102E10009C09FF1F9809FF1F9009FF1F2309FF1F2F
:102E20001C09FF1FA60BFF1FBC0BFF1FD40BFF1FAE
:102E3000FA210A4B0A4A49001A640A4A5A500A4AB5
:102E400004395A50094A08319A64094A5A50094AC1
:102E50005C315A50084ADA667047C0460000FF1FCE
:102E6000FD27FF1FF928FF1FAD28FF1FDD23FF1FD0
:102E70006D27FF1F7D1EFF1F511EFF1FF7B50B0C97
:102E8000FF270122009300233C001E001D009446F2
:102E9000019089B262469A401000084018413618E5
:102EA000B6B2FF2F02D1012E00D19FB2009802408E
:102EB0001A41AD18ADB2FF2C02D1012D00D19CB248
:102EC0000133102BE6D10320012E07D1012D04D1AF
:102ED000019B2401E4191C700138FEBD102EFCD1A9
:102EE0000238102DF9D00230F7E700008023F7B543
:102EF0009C46264B264F01932649274A274D284CAE
:102F0000284B02281AD1604638600868264E3040A7
:102F1000802636033043086001990978002909D1D9
:102F20001660224A2A60224A2260E02219689143F0
:102F3000A03A1BE08021C9021160F2E766463E60BC
:102F40000F68194E3E408027FF023E430E600199F4
:102F5000097800290DD1176001280ED1154A2A6081
:102F6000154A2260E02219689143C03A0A431A6068
:102F7000F7BD802189021160EEE7E0210F4A02438C
:102F80002A600F4A22601A688A43F0E74B0AFF1F43
:102F9000E0000340D80003409000034000000340DD
:102FA0005000034040000340FFFFE3FF0280063D66
:102FB000804508220180063D806608220080069830
:102FC00080550822F8B51E4B80261A680020140090
:102FD0003440324232D11A681A4F32431A60012209
:102FE0003B68063093433B6000F086FF0122164D9C
:102FF0002B681E432E603B680A2613433B608027E4
:10300000BF00124B1B683B4211D1013EF6B2FF2EAE
:1030100009D17E220E4B1C682B68E40B14409343AD
:1030200023432B6005E0082000F066FFE9E7002E4F
:10303000EFD180222B68600893432B60F8BDC04617
:10304000C4F000405CF0004018F0004068F0004020
:1030500060F0004010B500F0E7FE01215820034A5F
:1030600000F082FFFFF7AEFF10BDC046600AFF1FF1
:1030700010B578220021034800F0C6FF00F064FF7D
:10308000002010BD3867FF1F70B5040000F0CCFFB2
:1030900000230C200B4A010059438D18515C002974
:1030A0000DD0A14208D1012300246B7000F004FE72
:1030B00000F0DAFD200070BD01330A2BEBD11224A1
:1030C000F6E7C0463867FF1F70B5040000F0ACFF9C
:1030D000002319001D000D4A1078002806D0A042D8
:1030E0000CD1557001310C320A29F5D1002B0AD1CF
:1030F00000F02AFF00F0B8FD002070BD5078461E99
:10310000B0411B18EEE700F0D7FDF3E73867FF1F6B
:10311000F7B504000C20002384460E4D019267464B
:103120005F43E85D7E19A04212D000280BD10A4B04
:103130009C4662461B7808331370019B70707C5567
:103140007160B360FEBD01330A2BE8D10320F9E7BB
:103150000720F7E73867FF1F3467FF1F8020F8B5A7
:10316000484BC0051B68C1248360474BFF251A6884
:10317000012313434361454BA4001A68444B40218B
:103180001A60444B1A68444B1A60444B1A59AA43BC
:103190001A51C52292009E58AE4331438026995061
:1031A0009F583F49F6010F403E439E509E5880274E
:1031B0003602360A3043985080201A5900020A40DD
:1031C00002431A5104341A59364E3F0432408026C5
:1031D0003A431A511A5936061202120A32431A5148
:1031E00008341A5980260A4002431A51C322920019
:1031F0009F58B446AF4337439F509F58294E0F40C6
:1032000007439F509F583740802636043743802617
:103210009F509F5836063F023F0A37439F50C022B7
:103220001F59AF433A431A511A591202120A164350
:10323000C6221E5192009C58AC4365462C439C50BC
:103240009C5800250C4020439850C72080001A58F5
:10325000154C1140C02212020A431A50134B1B781E
:10326000DB08AB4201DC0020F8BD2378002B06D040
:10327000A368002B00D0984701350C34EEE71220EC
:10328000F2E7C0464443FF1F4043FF1FB0F0004039
:103290003067FF1FB4F000402C67FF1F00E100E023
:1032A000FF00FFFFFFFF00FF3867FF1F3467FF1FAE
:1032B000030010B51F2809D8072200201340072457
:1032C00004490A78A24313430B7010BD0023062063
:1032D000F5E7C0463467FF1F054B06491B780A68AF
:1032E00005485B0702401B0B134300200B6070472F
:1032F0003467FF1F1CF00040FFFFC1FF70B50C25B5
:10330000FFF7EAFF0A4B1C780A4BE4086543ED1807
:10331000002C01D1200070BD2B78002B06D06B68EB
:10332000002B00D09847013C0C3DF1E71220F2E75A
:103330003467FF1F2C67FF1F1FB5002102220B00FF
:1033400001910091052000F0A7FC02230B490A68B7
:103350001A42FCD120230393039B5A1E0392002B95
:10336000FAD1074A1368002BFCDA0B246C442000C6
:10337000012100F061FC207804B010BD90C800402D
:1033800000C8004013B504000A4B0193019B002BB9
:1033900001D1112016BDFFF7CFFF230003400442E7
:1033A00005D0052000F0A8FD019B013BEDE71800CA
:1033B000F0E7C046FFFFFF0707B500F035FE8022AB
:1033C0000821D205936A0191002B01D1073991623E
:1033D00002210C4A11600199481E01900029FAD17E
:1033E00003311160053101910199481E01900029B6
:1033F000FAD11160002B02D18022D205936200F035
:1034000033FC07BD00C00040F0B52D4C89B02378D7
:10341000002B4FD1FEF7D2FA02232A4F03903A68CD
:103420001A42FCD120230693069B5A1E0692002BBB
:10343000FAD1254E3368002BFCDA0120FFF7A2FFFA
:10344000011E02D0112009B0F0BD0300032201903B
:10345000009005AD9F2000F01FFC0321280000F024
:10346000EBFB02233A681A42FCD120230793079B07
:103470005A1E0792002BFAD13368002BFCDA012088
:10348000FFF780FF0028DDD10398FEF7ABFAAA789A
:103490006B7811041B020B4329780B436360130004
:1034A000113B0A49052B07D801239340A3600B6009
:1034B000012323700020C6E780231B03F6E7C046E4
:1034C0002C43FF1F90C8004000C800409808FF1F11
:1034D0001E4B30B55A6818781D4B85B0D318594229
:1034E0004B4101210093002300F09EFB194B1A4A27
:1034F00002259A6300221A6510325A658022C4217F
:103500009D65164B1648D202DA6789004258154B62
:1035100080241A4080231B0413434350642341201A
:103520000393E40500F006FA402000F003FA656218
:10353000039D6B1E0393002DFAD103236362FFF7F3
:103540003BFFA562FFF760FF05B030BD3843FF1FAA
:1035500095FFFEF700C80040050001FF04E100E010
:1035600000E100E0FFFF00FFF0B585B00700FEF7C7
:1035700025FA022305002D4C22681A42FCD1202393
:103580000093009B5A1E0092002BFAD1284E3368FC
:10359000002BFCDA0120FFF7F5FE002803D01124F0
:1035A000200005B0F0BD234B2360022322681A429D
:1035B000FCD120230193019B5A1E0192002BFAD1CA
:1035C0003368002BFCDA0120FFF7DCFE0028E6D18F
:1035D000194B1F60022322681A42FCD12023029358
:1035E000029B5A1E0292002BFAD13368002BFCDAA0
:1035F0000120FFF7C7FE0028D1D1104B2360022322
:1036000022681A42FCD120230393039B5A1E039283
:10361000002BFAD13368002BFCDA0120FFF7B2FE51
:10362000041EBCD12800FEF7DDF9B9E790C80040C0
:1036300000C8004001000006A8C800400180000149
:1036400010B50020FFF790FF10BD000010B5064B2D
:1036500018705960FFF73CFF00211320034AFFF761
:1036600057FD002010BDC0463843FF1FD134FF1F57
:10367000F0B5040085B003920291FEF79FF988220D
:1036800063035B0B52051A438023DB059D6A80238D
:10369000274F0092BA68002601901B039A420CD96A
:1036A000F82326001B041E401C4206D08022214B1A
:1036B00052025E6219680A431A60002D0BD100F0B5
:1036C000B3FC02221C4B1A608023DB055A62013ACC
:1036D0009A6200F0C9FA0023039A934220D1002D88
:1036E0000AD100F0A1FC144B03221D608023DB05EE
:1036F0005A629D6200F0B8FA8023BA681B039A42AE
:1037000008D9002E06D000220A4B0C495A621A68CA
:103710000A401A600198FEF765F9002005B0F0BD77
:10372000009A0299D2181278CA540133D4E7C046DD
:103730002C43FF1F00C8004000C00040FFFFFEFFF9
:10374000F0B587B0029103920400FEF737F90190BB
:1037500000F06AFC802302250122234EDB05356040
:103760005D629A6200F080FA204F3B682B42FCD1E8
:1037700020230493049B5A1E0492002BFAD11C4D63
:103780002B68002BFCDA0120FFF7FCFD002802D09B
:10379000112007B0F0BD2000039A029900F0BCFB95
:1037A000022304003A681A42FCD120230593059BAA
:1037B0005A1E0592002BFAD12B68002BFCDA01204F
:1037C000FFF7E0FD051EE3D100F02EFC802303226D
:1037D000DB0535605A629D6200F046FA0198FEF7FB
:1037E00001F9E0B2D5E7C04600C0004090C80040F3
:1037F00000C80040F0B5802489B00600FEF7DEF86E
:10380000E405A36A02250393029000F00DFC012356
:10381000304F3D606562A36200F026FA2E4C2368AB
:103820002B42FCD120230593059B5A1E0592002BA9
:10383000FAD12A4D2B68002BFCDA0120FFF7A2FDFC
:10384000002803D01124200009B0F0BD244B2360D0
:10385000022322681A42FCD120230693069B5A1E9B
:103860000692002BFAD12B68002BFCDA0120FFF71F
:1038700089FD021EE6D11B4B03211E60030001904F
:103880000090202000F008FA022322681A42FCD19E
:1038900020230793079B5A1E0792002BFAD12B680F
:1038A000002BFCDA0320FFF76DFD041ECAD100F0E7
:1038B000BBFB80230322DB053C605A629C6200F064
:1038C000D3F9039B002B01D1FFF776FD0298FEF799
:1038D00089F8B8E700C0004090C8004000C8004028
:1038E0000100000694C8004007B5000201910422BF
:1038F000000A01A9FFF724FF0EBD000073B5050003
:1039000005240B4AA3005B429B1819686B46DE1D19
:103910003000FFF7B3FA022804D133782B55013C6D
:10392000EFD276BD052CFCD00128FAD10230F8E7A1
:10393000140900111F2807D8012380228340D205D3
:1039400091680B43936070473F2808D80123802279
:1039500020388340D20551690B435361F3E75F2858
:10396000F1D80123802240388340D205116A0B43ED
:103970001362E8E71F2807D8012280218240C90589
:103980008B6893438B6070473F2808D801228021C1
:1039900020388240C9054B6993434B61F3E75F28A8
:1039A000F1D80122802140388240C9050B6A934337
:1039B0000B62E8E71F2810D880230200DB05153AC8
:1039C0001968012A06D820229143196019680A4310
:1039D0001A60704701228240F6E73F2811D8802301
:1039E0000200DB05353AD968032A06D81022914334
:1039F000D960D9680A43DA60EBE7012220388240B7
:103A0000F5E75F28E5D842238022181A413B83401E
:103A1000D205516A99435162516A0B435362D8E708
:103A200010B50400012813D1A022184992050B6893
:103A30005B015B0913430B60154B164A1968114073
:103A4000154A0A431A60402219680A431A6010BDD9
:103A50000028FCD101000A2000F016FA21000B20FA
:103A600000F012FAC0220A4B920019680A43402162
:103A70001A601A688A431A60B022044912060B6859
:103A80005B015B0913430B60E1E7C04614F00040A3
:103A90001CF000407F00FEFF80FD010072B6074A67
:103AA0001368013313600422054B1A600023054A92
:103AB00013608022D2055360FEE7C0467808FF1FDE
:103AC000C0F00040C4F0004005490B68002B05D150
:103AD000044A0A6004490A60044A13607047C046F9
:103AE000140AFF1F841E0000380AFF1FC4F00040A4
:103AF0000023034A1360034A1360034A13607047AC
:103B000054F0004040F1004044F1004002B47146DE
:103B100049084900095649008E4402BC7047C04616
:103B200002B4714649084900095C49008E4402BC50
:103B30007047C04603B47146490840004900095A1D
:103B400049008E4403BC704701B40248844601BC5E
:103B5000604700BF19FA000001B40248844601BC66
:103B6000604700BFE927000001B40248844601BC59
:103B7000604700BF8944000001B40248844601BC8C
:103B8000604700BF090E000001B40248844601BC32
:103B9000604700BF6D0B010001B40248844601BCC0
:103BA000604700BFE94C010001B40248844601BCF3
:103BB000604700BF0134010001B40248844601BCE3
:103BC000604700BFE512010001B40248844601BC11
:103BD000604700BF8552010001B40248844601BC21
:103BE000604700BF016C010001B40248844601BC7B
:103BF000604700BFE9F6000001B40248844601BCFA
:103C0000604700BFA9D8000001B40248844601BC47
:103C1000604700BFDD0C010001B40248844601BCCE
:103C2000604700BF8D11010001B40248844601BC09
:103C3000604700BFC56D010001B40248844601BC65
:103C4000604700BF3D71010001B40248844601BCD9
:103C5000604700BF85C1000001B40248844601BC32
:103C6000604700BF2144000001B40248844601BC03
:103C7000604700BF9DA9000001B40248844601BC12
:103C8000604700BFE9D4000001B40248844601BC8B
:103C9000604700BFC1F7000001B40248844601BC80
:103CA000604700BF496D010001B40248844601BC71
:103CB000604700BFC1A5000001B40248844601BCB2
:103CC000604700BF21A9000001B40248844601BC3E
:103CD000604700BF8937010001B40248844601BC37
:103CE000604700BFD9B0000001B40248844601BC5F
:103CF000604700BF6911010001B40248844601BC5D
:103D0000604700BFBD5C010001B40248844601BCAD
:103D1000604700BFB352010001B40248844601BCB1
:103D2000604700BF0D52010001B40248844601BC47
:103D3000604700BF71B0000001B40248844601BC76
:103D4000604700BFE90B010001B40248844601BC92
:103D5000604700BF51B8000001B40248844601BC6E
:103D6000604700BF5976010001B40248844601BC97
:103D7000604700BF0534010001B40248844601BC1D
:103D8000604700BF7997000001B40248844601BC37
:103D9000604700BF116E000001B40248844601BCB8
:103DA000604700BF2D6C010001B40248844601BC8D
:103DB000604700BFBD0B010001B40248844601BC4E
:103DC000604700BF53B9000001B40248844601BCFB
:103DD000604700BFCD0C010001B40248844601BC1D
:103DE000604700BFDD3F000001B40248844601BCCB
:103DF000604700BF4DF9000001B40248844601BC91
:103E0000604700BF9D6A000001B40248844601BCBF
:103E1000604700BF75F8000001B40248844601BC49
:103E2000604700BFC166010001B40248844601BC7E
:103E3000604700BFED68010001B40248844601BC40
:103E4000604700BFE9B5001101B40248844601BCD7
:103E5000604700BFCD4C010001B40248844601BC5C
:103E6000604700BF090E000001B40248844601BC4F
:103E7000604700BF8512010001B40248844601BCBE
:103E8000604700BFC9A9000001B40248844601BCD4
:103E9000604700BF65A2001101B40248844601BC1E
:103EA000604700BFDD0A010001B40248844601BC3E
:103EB000604700BF8D82000001B40248844601BC07
:103EC000604700BF156B010001B40248844601BC85
:103ED000604700BFF935010001B40248844601BCC7
:103EE000604700BFF9ED000001B40248844601BC00
:103EF000604700BF01D7000001B40248844601BCFE
:103F0000604700BF0189000001B40248844601BC3B
:103F1000604700BFEDA5000001B40248844601BC23
:103F2000604700BF9573010001B40248844601BC9C
:103F3000604700BFF90D010001B40248844601BC8E
:103F4000604700BFC115010001B40248844601BCAE
:103F5000604700BFADAE000001B40248844601BC1A
:103F6000604700BF6137010001B40248844601BCCC
:103F7000604700BF0167010001B40248844601BCEC
:103F8000604700BFED6B010001B40248844601BCEC
:103F9000604700BFF535010001B40248844601BC0A
:103FA000604700BF6DF6000001B40248844601BCC2
:103FB000604700BFC95C010001B40248844601BCEF
:103FC000604700BF0934010001B40248844601BCC7
:103FD000604700BFD1AE000001B40248844601BC76
:103FE000604700BFE917010001B40248844601BCE4
:103FF000604700BF7912010001B40248844601BC49
:10400000604700BF8914010001B40248844601BC26
:10401000604700BFB70E000001B40248844601BCEF
:10402000604700BF8B52010001B40248844601BCC6
:10403000604700BF75A9000001B40248844601BC76
:08404000604700BFD5440100F8
:10404800020000009ABE001101000000A0BC00118F
:104058000200000096BE0011010000008840FF1F0A
:1040680002000000A8BC001101000000C061FF1F91
:104078000200000094BE0011030000003461FF1F1D
:1040880012000000020000009ABE001101000000AA
:10409800E8BC00110200000096BE001101000000FB
:1040A800E5BC001102000000F2BC00110300000092
:1040B8006F61FF1F0200000094BE001103000000A2
:1040C8008461FF1F0200000096BE0011010000007D
:1040D800E4BC001102000000F0BC00110300000065
:1040E8004561FF1F0200000094BE0011030000009C
:1040F8006661FF1F020000009ABE00110100000067
:1041080028BD00110200000096BE00110100000049
:10411800D141FF1F020000003ABD0011010000005C
:1041280023BD00110200000096BE0011010000002E
:10413800D041FF1F0200000038BD0011010000003F
:104148008C61FF1F0200000096BE001101000000F4
:10415800CF41FF1F0200000036BD00110100000022
:1041680013BD00110200000096BE001101000000FE
:10417800CE41FF1F0200000034BD00110100000005
:104188000EBD00110200000096BE001101000000E3
:10419800CD41FF1F0200000032BD001101000000E8
:1041A80009BD00110200000096BE001101000000C8
:1041B800CC41FF1F0200000030BD001101000000CB
:1041C80004BD001102020202020200000000000009
:1041D8000D0C0000B14B0011774B001188BD001188
:1041E80090011D0018001800FFFF070102030405D5
:1041F80006020106000000000000000000000000A8
:1042080000000000000000000000000000000000A6
:1042180003000000020000009ABE00110100000027
:10422800A8BD00110200000096BE001101000000A8
:104238008C42FF1F02000000B2BD00110100000007
:10424800BA61FF1F0200000094BE001103000000C5
:104258002464FF1F0200000096BE00110100000048
:104268008C42FF1F02000000B0BD001101000000D9
:10427800BC61FF1F0200000094BE00110300000093
:104288001C64FF1F126C6C6C00000000005800409A
:10429800151600000001000000000111FFFF0000DA
:1042A8005048593600000000000000000B000500CF
:1042B800F0000000B4000028002800283075A00095
:1042C800A000A000A00000080008E001F000100015
:1042D8001000100010001000100050005000500096
:1042E80010001000D0070000000000000F000100BF
:1042F8000500307507001000010081FF0000000074
:10430800FF0000004D74001155720011E56F001197
:10431800FFFF0100FF000000699E0011E59B0011EE
:10432800FD9A0011000000000000000000000800D5
:10433800040000003B0001085902E0018821280020
:10434800FF000000020000009ABE001101000000FA
:1043580060BF00110200000096BE001101000000BD
:10436800C943FF1F0200000092BE001101000000B7
:10437800F067FF1F0200000096BE00110100000058
:10438800C843FF1F0200000090BE0011010000009A
:10439800C643FF1F0200000096BE00110100000086
:1043A800C443FF1F020000008EBE00110100000080
:1043B800BC43FF1F180018001D00900102000003F5
:1043C80002020000020000009ABE00110100000075
:1043D80074BF00110200000096BE00110100000029
:1043E8000C44FF1F020000008CBE001100000000FA
:1043F800000000000200000094BE0011030000004D
:064408001068FF1F20FFF9
:040000051FFF184180
:00000001FF
